S023000062696E2F6F70656E626C745F6F6C696D6578696E6F5F73746D33322E737265635A
S3150800000000500020410300088903000889030008FE
S315080000108903000889030008890300080000000016
S31508000020000000000000000000000000890300082E
S31508000030890300080000000089030008B14300088E
S315080000408903000889030008890300088903000852
S315080000508903000889030008890300088903000842
S315080000608903000889030008890300088903000832
S315080000708903000889030008890300088903000822
S315080000808903000889030008890300088903000812
S315080000908903000889030008890300088903000802
S315080000A089030008890300088903000889030008F2
S315080000B089030008890300088903000889030008E2
S315080000C089030008890300088903000889030008D2
S315080000D089030008890300088903000889030008C2
S315080000E08903000889030008890300080000000046
S315080000F000000000000000000000000000000000F2
S3110800010000000000000000005FF808F195
S3150800010C10B5054C237833B9044B13B10448AFF337
S3150800011C00800123237010BD40060020000000005B
S3150800012C1C660008084B10B51BB108490848AFF304
S3150800013C00800848036803B910BD074B002BFBD099
S3150800014CBDE81040184700BF000000004406002018
S3150800015C1C6600083C0600200000000070B50F4E17
S3150800016C0F4D761BB61018BF002405D0013455F870
S3150800017C043B9847A642F9D10A4E0B4D06F048FAAD
S3150800018C761BB61018BF002406D0013455F8043B6C
S3150800019C9847A642F9D170BD70BD00BF306E0008F5
S315080001AC306E0008386E0008306E000870B484078C
S315080001BC46D0541E002A41D0CDB2034602E0621E38
S315080001CCE4B3144603F8015B9A07F8D1032C2ED92D
S315080001DCCDB245EA05250F2C45EA054519D926461B
S315080001EC03F11002103E0F2E42F8105C42F80C5C1C
S315080001FC42F8085C42F8045C02F11002F2D8A4F149
S3150800020C100222F00F0204F00F041032032C1344D0
S3150800021C0DD91E462246043A032A46F8045BFAD838
S3150800022C221F22F003020432134404F003042CB1F7
S3150800023CC9B21C4403F8011BA342FBD170BC70471E
S3150800024C14460346C2E700BF024B13B1024800F03E
S3150800025C05B8704700000000750200080023014627
S3150800026C1A46184600F014B838B5074D074C2C1B1F
S3150800027CA41005D0013C55F8043D9847002CF9D13B
S3150800028CBDE8384006F0CAB93C6E0008386E00085E
S3150800029C2DE9F047254C064625688846D5F8484189
S315080002AC92469946C4B360681F2817DC411C76B180
S315080002BC04EB8003C3F888A0D4F888510122824045
S315080002CC1543022EC4F88851C3F808911ED0831C16
S315080002DC6160002044F82380BDE8F087144B03B313
S315080002EC4FF4C870AFF300800446D0B1D5F8483146
S315080002FC002784E888003846C5F848410121C4F827
S3150800030C8871C4F88C71002EE1D0D1E7D4F88C3101
S3150800031C1A43C4F88C21DAE705F5A674C5F84841E2
S3150800032CC1E74FF0FF30BDE8F08700BF3466000820
S3150800033C00000000002103E00B4B5B5843500431CE
S3150800034C0A480B4B42189A42F6D30A4A02E0002393
S3150800035C42F8043B084B9A42F9D300F01FFBFFF70F
S3150800036CFDFE00F019FA70473C6E000800000020EC
S3150800037C3C06002040060020981F0020FEE70000DF
S3150800038C12230B80004870474C04002004230B8072
S3150800039C004870474804002010B5044C0A46044827
S315080003AC214600F04FFD204610BD00BFD418002092
S315080003BC3866000810B5044C0A460448214600F075
S315080003CC41FD204610BD00BFD41800204866000821
S315080003DC10B5044C0A460448214600F033FD204665
S315080003EC10BD00BFD41800205C66000810B5044C7C
S315080003FC0A460448214600F025FD204610BD00BFDC
S3150800040CD41800206C66000810B5044C0A4604483B
S3150800041C214600F017FD204610BD00BFD418002059
S3150800042C7466000800F22C41D0F85C0400F078BD24
S3150800043C00EB4113D3F83C22D0F85C0400F0A0BDC5
S3150800044C00EB4113DA6BD0F85C0400F0CFBD00BFAB
S3150800045CD0F85C0400F052BE10B504460121D0F861
S3150800046C5C0400F035FED4F85C04BDE8104000F0DE
S3150800047C0FBE00BF10B5044602F028FFD4F85C0482
S3150800048C00F02AFEA36923B1024A136943F0060356
S3150800049C136110BD00ED00E008B5D0F85C0400F05F
S315080004AC25FEBDE8084002F013BF00BFF8B5214B86
S315080004BC214F0022C3F85C0404460826C0F82032F3
S315080004CC0225032118461F605E609D60D9609A61FB
S315080004DCDA611A6201F016FC20B140F213111748C2
S315080004EC03F07CFD002211461823D4F8200201F0F3
S315080004FCEDFB582300228021D4F8200201F0E6FBFC
S3150800050CC02300228121D4F8200201F0DFFB4FF42E
S3150800051C887300220121D4F8200201F0D7FBD4F805
S3150800052C20024FF480730022822101F0CFFB0020B9
S3150800053CF8BD00BFD41A0020005C00408C66000889
S3150800054C08B5D0F8200201F04DFC03289ABF024BDF
S3150800055C185C022008BD00BF9866000808B5D0F8DC
S3150800056C200201F061FC03289ABF024B185C02209A
S3150800057C08BD00BF9866000808B5D0F8200201F03F
S3150800058C6BFC03289ABF024B185C022008BD00BFFF
S3150800059C9866000810B51C46D0F820021346224669
S315080005AC01F0B0FC03289ABF014B185C022010BD61
S315080005BC9866000808B5D0F8200201F0C9FC032893
S315080005CC9ABF024B185C022008BD00BF986600084B
S315080005DC08B5D0F8200201F0DBFF03289ABF024BBE
S315080005EC185C022008BD00BF9866000808B5D0F84C
S315080005FC200201F0F9FF03289ABF024B185C02206F
S3150800060C08BD00BF986600080A06D0F8203204D444
S3150800061C03EB411393F82A02704701F07F0103EBB1
S3150800062C411393F82A00704708B5D0F8200201F058
S3150800063C55FC03289ABF024B185C022008BD00BF64
S3150800064C9866000808B5D0F8200201F0C5FC032806
S3150800065C9ABF024B185C022008BD00BF98660008BA
S3150800066C08B5D0F8200201F097FC03289ABF024B74
S3150800067C185C022008BD00BF9866000808B5D0F8BB
S3150800068C200201F0A1FC08BD012902D0002002F0CD
S3150800069C13BE084602F010BE20230380004870479C
S315080006AC600400200A230380004870478004002059
S315080006BC08B590F8FC31032B01D0002008BD03F0D7
S315080006CCBFFD002008BD00BF08B503F0B9FD00202A
S315080006DC08BD00BF08B5084603F0F2FD002008BDAA
S315080006EC10B504468121FFF765FF20460121FFF767
S315080006FC61FF002010BD00BF10B50446402302223E
S3150800070C8121FFF747FF2046402302220121FFF7EC
S3150800071C41FF20464023034A0121FFF7A1FF002091
S3150800072C10BD00BF341F002010B50C7814F0600FF4
S3150800073C07D14A7804460A2A05D00B2A14D0062A69
S3150800074C07D0002010BD01220E4900F04FF90020F9
S3150800075C10BD4A88120A212A0ED00B4917222046A8
S3150800076C00F044F9002010BD8B7813B9054A1360C4
S3150800077CE7E700F05BFBE4E7CA880449172A28BFB9
S3150800078C1722ECE75C06002069040020720400209E
S3150800079C00487047341F002008B502F011F9284AA2
S315080007AC136823F0070343F002031360136803F07E
S315080007BC0703022B03D06F21224803F00FFC224BB0
S315080007CC19461A6842F480321A600A681E4B90035E
S315080007DCFBD519465A6822F47C1242F4E8125A6080
S315080007EC1A6842F080721A600A68174B9201FBD598
S315080007FC19465A6822F0F0025A605A6822F4E062E6
S3150800080C42F480625A605A6822F460525A605A68F6
S3150800081C22F0030242F002025A604B680A4C03F0BB
S3150800082C0C03082BF9D1094800F076FC636823F40D
S3150800083C8003636003F06EFB03F07EFBFCE700BFEE
S3150800084C002002409C6600080010024000A24A04E0
S3150800085C334BF0B59A698DB042F001029A619A69E8
S3150800086C42F2200602F001020692069ADA692D4D2A
S3150800087C42F08052DA61DA69012402F0805205925C
S3150800088C059A9A6907A942F004029A619A6902279D
S3150800089C02F004020492049A9A69284642F0080265
S315080008AC9A619A6902F008020392039A9A6942F0CD
S315080008BC10029A619A6902F010020292029A9A69D7
S315080008CC42F020029A619A6902F020020192019A7A
S315080008DCDA6942F40002DA61DB69079603F400036D
S315080008EC00930026009B089409970A9601F06CF968
S315080008FC20220D4B6A6107A90C480793089409979F
S3150800090C0A9601F061F940F20112082307A9284654
S3150800091C0B940792089301F057F90DB0F0BD00BF80
S3150800092C001002400008014010001004001001409D
S3150800093C08B5154801F0F0F8144801F0EDF814481C
S3150800094C01F0EAF8134801F0E7F8134BDA6922F4D8
S3150800095C0002DA619A6922F020029A619A6922F0F9
S3150800096C10029A619A6922F008029A619A6922F031
S3150800097C04029A61DA6922F08052DA619A6922F0E5
S3150800098C01029A6108BD00BF001401400010014025
S3150800099C000C01400008014000100240104B10B436
S315080009AC1968104A41F00101196059680E480A4045
S315080009BC5A601A684FF41F0422F0847222F48032AB
S315080009CC1A601A684FF0006122F480221A605A687D
S315080009DC22F4FE025A609C60816010BC704700BF0E
S315080009EC001002400000FFF800ED00E038B5134691
S315080009FC02250A468361C361C0F8F4510021FFF74A
S31508000A0C21FE002038BD00BF08B513460A46002152
S31508000A1CFFF718FE002008BD08B513460A46002144
S31508000A2CFFF71EFE002008BD08B504220023C0F8F7
S31508000A3CF42119461A46FFF705FE002008BD00BF2B
S31508000A4C08B505220023C0F8F42119461A46FFF703
S31508000A5C07FE002008BD00BF30B54B7883B00D46A5
S31508000A6C0446092B0BD8DFE803F035490A590A0561
S31508000A7C660A7D158B8813B9CB88002B7FD080210D
S31508000A8C2046FFF7A5FD20460021FFF7A1FD002013
S31508000A9C03B030BD8978974D01292970EFD890F8A5
S31508000AACFC31022B00F08980032BE8D1002900F0D9
S31508000ABC16814168012909D0C9B200F029FA2978AA
S31508000ACC2046616000F01AFA0228D8D02046FFF7B3
S31508000ADCABFFDCE790F8FC310122023B93424FF066
S31508000AEC0301CCD8D0F80432C26003B1C16002222B
S31508000AFC04F10C012046FFF779FFC8E790F8FC31A2
S31508000B0C023B012BBBD84B88012BC0D1D0F8143231
S31508000B1C00229B68C0F804229847D7E74B88012B1C
S31508000B2CB5D1D0F81422C0F80432936898472046F9
S31508000B3CFFF77AFFABE74A88130A013B062B9ED8C8
S31508000B4C01A151F823F000BF370C0008590C000816
S31508000B5C470C00088B0A00088B0A0008210C0008B1
S31508000B6CE10B0008CA88012A89D190F8FC31022BBE
S31508000B7C1CD0032B83D1011DFFF738FF87E790F8AC
S31508000B8CFC318D78032B05F07F053FF478AF80F8A0
S31508000B9CFE512946FFF748FD2046FFF745FF002D75
S31508000BAC00F09080022384F8FC3170E7014600239C
S31508000BBC41F8083FFFF71AFF69E7002986D001219B
S31508000BCC0323416080F8FC3100F098F902287FF481
S31508000BDC7DAF54E7037C002B7FF451AFD0F8143269
S31508000BEC0DF106001B6B984707234370BDF80630BA
S31508000BFC002B3FF44CAFEA88002A3FF448AF9342E7
S31508000C0C28BF134601461A462046ADF80630FFF7AC
S31508000C1CEDFE3CE7037C002B7FF431AFD0F81432A1
S31508000C2C0DF106005B6B9847E0E7D0F810320DF132
S31508000C3C06011B68007C9847D8E7D2B2052A3FF60E
S31508000C4C1EAFDFE802F0271F170F372F037C002B88
S31508000C5C3CD1D0F814320DF106009B6A9847022352
S31508000C6C4370C3E7D0F810320DF106011B69007CFE
S31508000C7C9847BBE7D0F810320DF10601DB68007C0B
S31508000C8C9847B3E7D0F810320DF106019B68007C43
S31508000C9C9847ABE7D0F810320DF106015B68007C7B
S31508000CAC9847A3E7D0F810320DF106019B69007C32
S31508000CBC98479BE7D0F810320DF106015B69007C6A
S31508000CCC984793E7012384F8FC31E0E6D0F8143210
S31508000CDC0DF10600DB6A98470223437086E7022368
S31508000CEC416080F8FC3100F013F92046FFF79CFEB2
S31508000CFCCDE600BF6006002038B590F8FC310446F6
S31508000D0C032B03D10B790D46012B08D98021FFF74C
S31508000D1C5FFC20460021FFF75BFC002038BDD0F8AD
S31508000D2C14329B689847EB88002BF6D12046FFF7C0
S31508000D3C7BFEF2E770B50B788A8803F06003202BEC
S31508000D4C054657D04B780C46012BD6B234D019D35E
S31508000D5C032B15D190F8FC31022B31D0032B40D143
S31508000D6C4B8823B9730602D03146FFF731FCD5F808
S31508000D7C143221469B68284698472846FFF754FEA6
S31508000D8C002070BD90F8FC31022B19D0032B28D10A
S31508000D9C06F07F04130600EB041431464CBF1434DA
S31508000DAC04F58274FFF730FC48BB206021462846C0
S31508000DBC0222FFF71BFEE3E790F8FC31022B05D164
S31508000DCC7206DDD03146FFF703FCD9E7032B08D1B1
S31508000DDC4B88002BD4D17106CFD03146FFF706FCD1
S31508000DECC5E78021FFF7F4FB28460021FFF7F0FB47
S31508000DFC002070BDD0F814329B689847C0E70123D1
S31508000E0C2360D3E70B7803704B784370CA788B78DA
S31508000E1C03EB022343804A790B7903EB0223838085
S31508000E2CCA798B7903EB0223C380704710B5044645
S31508000E3C8021FFF7CDFB2046BDE810400021FFF7C7
S31508000E4CC7BB00BF00B3037830B4F3B10446002324
S31508000E5C14F8015F0133DBB2002DF9D15B000233C4
S31508000E6CDCB2032513800C704D7004785CB1022338
S31508000E7C00255A1CD2B2CC548D5410F8014F0233AB
S31508000E8CDBB2002CF5D130BC704702242346E8E7C8
S31508000E9C88B108B5D0F8143213B10023C0F814324F
S31508000EAC09B1C0F810120123027080F8FC31FFF763
S31508000EBCFDFA002008BD0220704700BF10B5044695
S31508000ECC0122D0F8143280F8FC215B680179984726
S31508000EDC2046FFF751FB2046FFF732FB002010BDDA
S31508000EEC19B1C0F81412002070470220704700BFD1
S31508000EFC08B5FFF733FB002008BD00BF08B5D0F8CE
S31508000F0C143213B11B68984708B1022008BD08BDF6
S31508000F1C08B5D0F814325B689847002008BD00BFA6
S31508000F2C38B5044600F502752846FFF76BFF94F8AA
S31508000F3C08120120B4F80E2201F01F038342C4F8EC
S31508000F4CF401C4F8F82115D00ED3022B06D001F003
S31508000F5C80012046FFF73CFB002038BD2946204679
S31508000F6CFFF7E8FE002038BD29462046FFF774FD3A
S31508000F7C002038BD29462046FFF7BEFE002038BDA6
S31508000F8C10B5044631B91346D0F8F421032A0CD00F
S31508000F9C002010BDD0F814329B69002BF8D090F8BD
S31508000FACFC21032AF4D19847F2E7D0F80C11D0F8B3
S31508000FBC102191420CD8D0F814321B691BB190F849
S31508000FCCFC21032A0FD02046FFF72EFD002010BD6A
S31508000FDC891A8A4228BF0A46C0F80C1192B21946D9
S31508000FECFFF71AFDD4E79847EDE700BF70B504463E
S31508000FFC51B91346D0F8F421022A15D094F80032C8
S3150800100C012B0CD0002070BDD0F814325B69002B74
S3150800101CF8D090F8FC21032AF4D19847F2E700237C
S3150800102C84F80032002070BDC669026A964223D83D
S3150800103C8369B3FBF2F502FB15358DB99A420FD8C5
S3150800104CD0F8F82193420BD22A46FFF7DDFCC4F8F8
S3150800105CF8512B462A4629462046FFF701FBCDE7D1
S3150800106CD4F81432DB681BB194F8FC21032A0BD094
S3150800107C2046FFF7E5FCC1E7B21A0D46C2611946D0
S3150800108C92B2FFF7C1FCE4E720469847F0E700BFA9
S3150800109C38B5402304461D4600221146FFF77AFA56
S315080010AC2B460022C4F8105120468021FFF772FA0D
S315080010BCD4F818320122256284F8FC212BB1D4F815
S315080010CC143221795B6820469847002038BD00BF4A
S315080010DC01740020704700BF90F8FC21042380F8A7
S315080010ECFD2180F8FC310020704700BF034690F8BC
S315080010FCFD21002083F8FC21704700BF90F8FC21E5
S3150800110C032A01D00020704708B5D0F81432DB69E1
S3150800111C03B19847002008BD014B1860704700BF03
S3150800112CC404002084B001A880E80E0004B0002096
S3150800113C704700BF0246B0F8403000209BB243F41B
S3150800114C3F43A2F84030704744F2FF210246B0F8FC
S3150800115C403000200B40A2F8403070470020704702
S3150800116C84B070B4044601250020A4F84050A4F8B5
S3150800117C4000A4F84400A4F85000B4F8405004AE5B
S3150800118CADB245F43F45A4F8405086E80E0070BC55
S3150800119C04B07047CB7830B4032B10D8DFE813F0C3
S315080011AC7501680104005B010A7830F8223023F4D3
S315080011BCEC4323F070031B041B0C20F822300C782C
S315080011CC30F8243044F4004223F0F0031B051B0DC1
S315080011DC42F08002134320F824308B7A002B37D147
S315080011EC4B78002B00F0EE80B0F850300C788A88DB
S315080011FC9BB203EBC403520800EB43035200C3F83B
S3150800120C00240C7830F8243000EB84025D060ED5E9
S3150800121C30F8243023F0F0031B051B0D43F4004370
S3150800122C43F0C00320F824300A7800EB82021388B6
S3150800123C002023F4E04323F040031B041B0C83F02B
S3150800124C200343F4004343F08003138030BC7047FB
S3150800125C0A7800F5806430F8223023F4F8731B05FD
S3150800126C1B0D43F4014343F0800320F82230B0F8F9
S3150800127C5030CD880A789BB26D0803EBC2026D001C
S3150800128CB0F8503044F812500A890D789BB20433E2
S3150800129C520803EBC503520044F813204B780C781C
S315080012AC002B4FD130F8243000EB84025D040ED5A8
S315080012BC30F8243023F0F0031B051B0D43F4404390
S315080012CC43F0800320F824300A7800EB8202138856
S315080012DC5B060CD5138823F0F0031B051B0D43F492
S315080012EC004343F0C00313800A7800EB820213888C
S315080012FC30BC23F0F0031B051B0D43F4004343F0ED
S3150800130CC00313800A7830F8223023F4804323F084
S3150800131C70031B041B0C83F4405343F4004343F043
S3150800132C800320F822300A7830F8223023F0C003E4
S3150800133C1B051B0D43F4004343F0800320F82230B1
S3150800134C0020704730F8243000EB84025D040ED57B
S3150800135C30F8243023F0F0031B051B0D43F44043EF
S3150800136C43F0800320F824300A7800EB82021388B5
S3150800137C5B0600F1978030BC138823F0F0031B053D
S3150800138C1B0D43F4404343F0800313800A7830F86E
S3150800139C223023F0C0031B051B0D43F4004343F016
S315080013AC800320F822300A7830F8223023F0F00334
S315080013BC9B049B0C43F4004343F0800320F8223033
S315080013CC00207047B0F850308C880A789BB20433EA
S315080013DC640803EBC202640000F58065B0F850306F
S315080013EC45F812400C690A789BB206333E2C03EB7F
S315080013FCC20365D8C4F34F02E40744BF013292B264
S3150800140C920292B245F813200C7830F8243000EB8F
S3150800141C84025B040ED530F8243023F0F0031B0548
S3150800142C1B0D43F4404343F0800320F824300A781C
S3150800143C00EB82021388002023F4804323F0700308
S3150800144C1B041B0C83F4405343F4004343F0800302
S3150800145C138030BC70470A7830F822309BB223F4DC
S3150800146CEC4323F0700343F4C06320F82230A6E65D
S3150800147C0A7830F822309BB223F4EC4323F070033D
S3150800148C43F4806320F8223099E60A7830F8223043
S3150800149C9BB223F4EC4323F0700343F4007320F857
S315080014AC22308CE6138823F0F0031B051B0D43F43E
S315080014BC004343F0C00313800A7800EB82025AE714
S315080014CCC4F34F12E40604BF02F1FF3292B26FEA7C
S315080014DCC2626FEA524292B245F8132094E700BFF3
S315080014EC8B7A10B433BB4B780C78002B00F0B18098
S315080014FC30F8243000EB84025B060ED530F8243025
S3150800150C23F0F0031B051B0D43F4004343F0C00303
S3150800151C20F824300A7800EB82021388002023F086
S3150800152CC0031B051B0D43F4004343F080031380D3
S3150800153C10BC70474B780C78002B4BD130F8243004
S3150800154C00EB84025B040ED530F8243023F0F0034C
S3150800155C1B051B0D43F4404343F0800320F824304D
S3150800156C0A7800EB820213885C060CD5138823F0E4
S3150800157CF0031B051B0D43F4004343F0C003138013
S3150800158C0A7800EB8202138810BC23F0F0031B05C3
S3150800159C1B0D43F4004343F0C00313800A7830F85C
S315080015AC223023F0F0039B049B0C43F4004343F0D6
S315080015BC800320F822300A7830F8223023F0C00352
S315080015CC1B051B0D43F4004343F0800320F822301F
S315080015DC0020704730F8243000EB84025B040ED5EB
S315080015EC30F8243023F0F0031B051B0D43F440435D
S315080015FC43F0800320F824300A7800EB8202138823
S3150800160C5B0648D4138810BC23F0F0031B051B0D8E
S3150800161C43F4404343F0800313800A7830F82230B1
S3150800162C23F0C0031B051B0D43F4004343F0800352
S3150800163C20F822300A7830F8223023F0F0039B0485
S3150800164C9B0C43F4004343F0800320F8223000201F
S3150800165C704730F8243000EB84025B040ED530F862
S3150800166C243023F0F0031B051B0D43F4404343F0D1
S3150800167C800320F824300A7800EB820213880020B5
S3150800168C23F0F0039B049B0C43F4004343F08003C4
S3150800169C138010BC7047138823F0F0031B051B0D31
S315080016AC43F4004343F0C00313800A7800EB82022C
S315080016BCA8E700BF4A78F0B4012A70D08B690C6988
S315080016CCA34232D800248C618C7A002C33D1B0F822
S315080016DC50200C7892B206323E2B02EBC40200F56F
S315080016EC806540F29780C3F34F14DE0604BF04F1FD
S315080016FCFF34A4B26FEAC4646FEA5444A4B245F842
S3150800170C12400A78F0BC30F8223023F4804323F0D8
S3150800171C70031B041B0C83F4405343F4004343F03F
S3150800172C800320F82230002070471B1B8B61234650
S3150800173C8C7A002CCBD0002AE3D1B0F850200C7848
S3150800174C92B202323E2B02EBC40200F5806640F2DE
S3150800175CA38013F01F07C3F34F1412BF254604F1D9
S3150800176CFF35ADB26FEAC5656FEA5545ADB246F8B9
S3150800177C12504A78002A40F0C980B0F850300A78DE
S3150800178C9BB2063303EBC2030FB9013CA4B26FEA52
S3150800179CC4626FEA524292B246F81320B1E78C69DA
S315080017AC0B699C4241D800238B618B7A002B42D162
S315080017BCA3B28A88013300EB42025B104D6918BF4D
S315080017CC02F2044207D035F8026B013B22F8046C8E
S315080017DC02F10402F7D1B0F850300A789BB2023302
S315080017EC03EBC20300EB4303C3F800440A78F0BCCE
S315080017FC30F8223023F4E04323F040031B041B0C7F
S3150800180C83F0300343F4004343F0800320F822307E
S3150800181C00207047C3F34F04DB0744BF0134A4B25E
S3150800182CA402A4B245F812406BE7E41A8C611C4674
S3150800183C8B7A002BBCD00E7830F826305F0648D54C
S3150800184CB0F8505000F58063ADB2023505EBC60210
S3150800185C0E8943F81240A2B20132521003EB460627
S3150800186C4C6918BF002306D034F8025B26F82350BF
S3150800187C01339342F8D14B78002B36D10A7830F8DD
S3150800188C223023F0F0031B051B0D43F4004343F0F1
S3150800189CC00320F82230A9E713F00107C3F34F045D
S315080018AC0EBF2546651CADB2AD02ADB246F8125058
S315080018BC4A785ABBB0F850300A789BB2063303EB19
S315080018CCC2030FB10134A4B2A402A4B246F8134061
S315080018DC17E7B0F8502000F5806392B2023202EB9B
S315080018ECC602CE8843F81240B5E7012B7FF47EAFCB
S315080018FC0A7830F8223023F0F0031B051B0D43F44D
S3150800190C404343F0800320F822306FE7012A7FF426
S3150800191CF8AEB0F850200C7892B2023202EBC40240
S3150800192C46F81230EDE600BF0A782AB34B788BB925
S3150800193C30F8223023F4804323F070031B041B0C6D
S3150800194C83F4805343F4004343F0800320F8223099
S3150800195C0020704730F8223023F4E04323F040038C
S3150800196C1B041B0C83F0100343F4004343F0800361
S3150800197C20F822300020704703889BB223F480435A
S3150800198C23F0400383F4805383F0100343F400439D
S3150800199C43F0800303800020704700BF4B7810B4D7
S315080019AC0C782BB330F8243000EB84025B060ED58A
S315080019BC30F8243023F0F0031B051B0D43F40043C9
S315080019CC43F0C00320F824300A7800EB820213880F
S315080019DC002023F4E04323F040031B041B0C83F084
S315080019EC300343F4004343F08003138010BC704764
S315080019FC30F8243000EB84025B040ED530F8243022
S31508001A0C23F0F0031B051B0D43F4404343F08003FE
S31508001A1C20F824300A7800EB82021388002023F47D
S31508001A2C804323F070031B041B0C83F4405343F4CC
S31508001A3C004343F08003138010BC70470346002212
S31508001A4C01200321A3F84000A3F844201046A3F86C
S31508001A5C4010704711B98023A0F84C30002070470D
S31508001A6C0020704700207047B0F8440080B27047D9
S31508001A7C00207047013300F580605B1000EB4202D2
S31508001A8C09D030B4002431F8025B22F82450013412
S31508001A9CA342F8D130BC7047013300F580605B1067
S31508001AAC00EB420205D052F8040B013B21F8020B5D
S31508001ABCF9D1704703685B062BD4024670B44B68A1
S31508001ACC0C688D681C43CB6808692C431C434D690C
S31508001ADC8E692043136840EA0504C86934430E6AC4
S31508001AEC204323F47F43304323F0BF03034313609F
S31508001AFC5368B6F5005F23F0040343EA15435360B5
S31508001B0C02D070BC012070478B8C0120136170BC0D
S31508001B1C70470020704700BF264B984219D0264BB9
S31508001B2C984222D0254B98422BD0254B984234D03C
S31508001B3C244B984201D00020704703F57843DA68A5
S31508001B4C012042F04002DA60DA6822F04002DA60DC
S31508001B5C704703F58433DA68012042F00402DA6030
S31508001B6CDA6822F00402DA60704703F58233DA6821
S31508001B7C012042F00802DA60DA6822F00802DA601C
S31508001B8C704703F58033DA68012042F01002DA60F8
S31508001B9CDA6822F01002DA60704703F57C43DA68DB
S31508001BAC012042F02002DA60DA6822F02002DA60BC
S31508001BBC704700BF00080140000C014000100140AE
S31508001BCC00140140001801402DE9F04F0D68C5F3CB
S31508001BDC0F2595FAA5F4B4FA84F435FA04F371D002
S31508001BEC40F2011C4FF00F0E4FF001190123A340D0
S31508001BFC2B4263D0072C85BFA4F1080309FA03F31B
S31508001C0C0CFA04F343F080631E0E93FAA3FABAFA9D
S31508001C1C8AFA93FAA3F8B8FA88F84A6887594FEA01
S31508001C2C8A0A4FEA88080EFA0AFA27EA0A0A02FA10
S31508001C3C08F24AEA02028251D0F80CA01A0A92FA61
S31508001C4CA2F8B8FA88FB2AEA020A0F694A6807FA60
S31508001C5C0BF822F008024AEA0808012AC0F80C8098
S31508001C6C2CD193FAA3FABAFA8AFA93FAA3F8B8FA21
S31508001C7C88F803274FEA8A0A8A6807FA0AFA8759FC
S31508001C8C4FEA880827EA0A0A02FA08F24AEA02021E
S31508001C9C825193FAA3F8B8FA88F893FAA3F3B3FA2D
S31508001CAC83F304274FEA880807FA08F8CF689B00DD
S31508001CBC22EA080207FA03F31A438251013435FA69
S31508001CCC04F393D10120BDE8F08F00BF11F0800F0B
S31508001CDC0CD001F07F0100EB4110283062B1190CD1
S31508001CEC0122C380018182720020704700EB4110EB
S31508001CFC00F50A70002AF2D18272838000207047A0
S31508001D0C704700BF002869D0F0B590F8293487B021
S31508001D1C044603F0FF02002B5BD02546032384F808
S31508001D2C29342068FFF710FA55F810EB6F462E4643
S31508001D3C0FCE0FC73368261D3B6096E80E0070461B
S31508001D4CFFF7F0F900212068FFF708FA002108468A
S31508001D5C23462246012782F82810918601310F293D
S31508001D6C82F8297082F82B009063D063106402F114
S31508001D7C2002F0D10022114683F828229A860132D5
S31508001D8C0F2A83F8291283F82B12C3F83812C3F8D2
S31508001D9C3C12C3F840124FF0000703F12003EBD1B5
S31508001DACEE460FCDD4F800C0AEE80F002B6860469F
S31508001DBCCEF8003096E80E00FFF7D2F9012384F826
S31508001DCC2470206884F82934FFF74CFE384607B08F
S31508001DDCF0BD80F82824FFF793FF9EE70120704793
S31508001DEC704700BFF0B190F828340322012B10B5C8
S31508001DFC044680F829240ED0012380F8283400687C
S31508001E0CFFF7A2F92068FFF719FE2068FFF72AFEEC
S31508001E1C002384F828342046FFF7E2FF002084F8D4
S31508001E2C290410BD0120704790F82824012A01D1F5
S31508001E3C0220704710B50446012180F82814FEF7D5
S31508001E4C23FC2068FFF70CFE2068FFF773F90020C7
S31508001E5C84F8280410BD00BF90F82834012B01D152
S31508001E6C0220704710B50446012380F82834006810
S31508001E7CFFF76AF92068FFF7E1FD2068FFF7F2FD26
S31508001E8C002084F8280410BD90F82824012A01D1D2
S31508001E9C0220704710B50446012180F82814FEF775
S31508001EACF3FB2068FFF7DCFD002084F8280410BD3E
S31508001EBC90F82824012A01D10220704710B504464F
S31508001ECC012380F828340021FEF7DEFB2068FFF793
S31508001EDCC9FD002084F8280410BD00BF90F82824FA
S31508001EEC012A01D10220704710B50446012284F854
S31508001EFC241080F828240068FFF7ACFD002084F82D
S31508001F0C280410BD38B54CB2002C1ADB0D4600EB74
S31508001F1C411101F50A71E40F4C700D70CB7090F8F5
S31508001F2C28340A61012B01D1022038BD044601234D
S31508001F3C80F828340068FFF72DF9002084F8280467
S31508001F4C38BD01F07F0500EB45112831E3E700BFEA
S31508001F5C4BB2002B19DB0A4600EB411101F50A714D
S31508001F6CDB0F4B700A7090F82834012B01D1022034
S31508001F7C704710B50446012380F828340068FFF72B
S31508001F8CAFFA002084F8280410BD01F07F0200EB9C
S31508001F9C42112831E4E700BF70B501F07F014D010D
S31508001FAC4419002684F82812C4F83C22C4F8403296
S31508001FBCC4F8446284F8296205F50A71014400687C
S31508001FCCFFF778FB304670BD01F00F0100EB4110AE
S31508001FDCB0F84402704700BFF8B501F07F014D0117
S31508001FEC44190026012784F82810E263236484F830
S31508001FFC2970666405F1280101440068FFF75AFB4D
S3150800200C3046F8BD2DE9F043044683B00068FFF767
S3150800201C2BFD020444D42068FFF726FD460500F183
S3150800202C09822068FFF720FD10F4804F206807D03E
S3150800203CB0F8443023F480431B041B0CA0F844303E
S3150800204CFFF712FD10F4005F206807D0B0F8443093
S3150800205C23F400531B041B0CA0F84430FFF704FDB3
S3150800206CC50400F1C9812068FFF7FEFC000500F1E4
S3150800207CA2812068FFF7F8FC820500F18F812068A1
S3150800208CFFF7F2FCC30508D52268B2F8443023F4EE
S3150800209C80731B041B0CA2F8443003B0BDE8F08314
S315080020AC00232068ADF8043004F22C46ADF806304F
S315080020BCB0F844309BB21F04ADF80430ACD5BDF86B
S315080020CC042012F00F075BD1BDF80410038801F049
S315080020DC100189B2002900F0A0809BB2ADF8063039
S315080020ECBDF806301B0500F13881BDF806301F0413
S315080020FCDED5038823F070031B051B0D0380B0F88F
S3150800210C503094F828229BB2063303EBC20300EB3B
S3150800211C4303D3F80034C3F30903C4F84432002B41
S3150800212C40F01A8200212046FEF782F92068D4F87E
S3150800213C3852B0F850303E2D9BB200F5806103F151
S3150800214C060340F2DA81C5F34F12ED0604BF02F11D
S3150800215CFF3292B26FEAC2626FEA524292B241F809
S3150800216C1320038823F4804323F070031B041B0CF1
S3150800217C83F4405343F4004343F08003038097E70A
S3150800218C30F827309BB2ADF80630BDF806301D0482
S3150800219C72D4BDF806301A068AD530F827307D0178
S315080021AC23F4E14323F070031B041B0C20F827309F
S315080021BC04EB050E9EF83230002B40F0AB80B0F8DD
S315080021CC50309EF828209BB2023303EBC20300F56D
S315080021DC806151F8133004EB4712C3F309035364B7
S315080021EC002B40F08081B0F85030254495F8282013
S315080021FC9BB2023303EBC20351F81310EA6BC1F31B
S3150800220C09012B6C0A446964EA6395F82810204680
S3150800221C73BBFEF715F920684AE723F4E14323F06C
S3150800222C70031B041B0CE26B0380B0F8503094F857
S3150800223C28509BB2023303EBC50300EB4300D0F8DE
S3150800224C00342046C3F309031A446364E263FEF7B9
S3150800225CF7F894F824306BB1236C5BB994F8242006
S3150800226C206842F08002A0F84C2084F824301FE73E
S3150800227CFFF7B2FE20681BE730F827307D0123F004
S3150800228C70031B051B0D20F8273004EB050999F87C
S3150800229C3232002B00F0EC8099F828E230F82E3018
S315080022AC00EB8E02590440F13381B0F8501089B214
S315080022BC023101EBCE0300EB4303D3F80034C3F32E
S315080022CC0908B8F1000F40F05F81138823F0F0037A
S315080022DC1B051B0D43F4004343F0C003138061191F
S315080022ECD1F84402D1F83C22D1F840324044424459
S315080022FCC1F84402C1F83C2223B1D1F83802804512
S3150800230C80F023812544204695F82812FEF790F88C
S3150800231C20683EE79EF828C030F82C305B0640F162
S3150800232CC180B0F8501004EB471289B2023101EBA8
S3150800233CCC0300F5806151F81330C3F309035364D9
S3150800234C002B00F0C080DEF83C10BEF82E20FFF7FC
S3150800235C91FB206800F58061B5E0B0F8503094F830
S3150800236C28229BB2063303EBC20300EB4303D3F8D4
S3150800237C0034B4F82C22C3F30903C4F844323146AA
S3150800238CFFF78AFB22682046138823F070031B0587
S3150800239C1B0D1380FEF746F8206889E6226820464E
S315080023ACB2F8443023F400731B041B0CA2F8443017
S315080023BCFEF74EF863E62368B3F84020184692B247
S315080023CC42F00802A3F84020B3F8442022F4006235
S315080023DC1204120CA3F84420B3F8402092B242F02F
S315080023EC0402A3F84020FFF73FFBC1043FF541AEBA
S315080023FC2046FEF73FF83CE622682046B2F8403005
S3150800240C23F004031B041B0CA2F84030B2F840302E
S3150800241C23F008031B041B0CA2F84030FEF73CF80B
S3150800242C2068B0F8443023F480531B041B0CA0F826
S3150800243C443019E622682046B2F8443023F4806307
S3150800244C1B041B0CA2F84430FEF706F894F8283443
S3150800245C012B3FF4E6AD0025012384F8283484F8D3
S3150800246C245029462068FFF7F5FA84F82854D8E54D
S3150800247CB0F8503099F828229BB2063303EBC20306
S3150800248C00EB4303D3F80034C3F30908B8F1000F83
S3150800249C3FF425AF4346B9F82C22D9F83C12FFF77E
S315080024ACFBFA1CE7B0F8503000F580619BB2063396
S315080024BC03EBCC0351F8133004EB4712C3F30903AF
S315080024CC5364002B56D1631993F8282030F8223020
S315080024DC23F0F0031B051B0D43F4404343F0800324
S315080024EC20F822307FE6DEF83C10BEF82C20FFF7E9
S315080024FCC1FA206800F5806175E6C5F34F02EF074F
S3150800250C44BF013292B2920292B241F8132028E6E5
S3150800251CB0F850309BB2063303EBCE0300EB430303
S3150800252CD3F80034C3F30908B8F1000F3FF4CDAE65
S3150800253C4346B9F83022D9F83C12FFF7ADFA99F8A8
S3150800254C2822236803EB8202BFE691F8281220465C
S3150800255CFFF722FD20681CE6B4F82C22D4F83C12AE
S3150800256CFFF79AFAD4F83C22D4F844321344C4F848
S3150800257C3C32D7E5DEF83C10BEF83020FFF77AFA85
S3150800258C206800F580619EE74346B9F82E22D2E70B
S3150800259C38B54BB2002B1ADB0D4600EB411101F591
S315080025AC0A71DB0F01224B700D708A7090F8283473
S315080025BC934201D1022038BD044680F828240068CD
S315080025CCFFF7B2F94DB1002084F8280438BD01F0A4
S315080025DC7F0500EB45112831E3E704F22C4120680E
S315080025ECFFF746FAEFE700BF38B54BB2002B1ADBFC
S315080025FC0A4600EB411101F50A71DB0F00254B70F9
S3150800260C0A708D7090F82834012B01D1022038BD40
S3150800261C0446012380F828340068FFF7BFF984F8CC
S3150800262C2854284638BD01F07F0200EB42112831A8
S3150800263CE3E700BF2DE9F8432E4E337E012B43D03A
S3150800264C03680122022B8146884632764CF25030BA
S3150800265C32D000F09BF890BB4FF0FF33C8F800302F
S3150800266CD9F80850D9F80C3005EB83239D4226D2AD
S3150800267C0746214C09E0D9F80C20D9F8083005F59D
S3150800268C806503EB8223AB421AD9F76123694CF2B6
S3150800269C503043F0020323616561236943F040031C
S315080026AC236100F073F8236923F0020323610028E1
S315080026BCE1D0C8F8005003E000F068F838B1012002
S315080026CC00233376BDE8F8830220BDE8F8830A4C6C
S315080026DCF06123694CF2503043F0040323612369FB
S315080026EC43F04003236100F051F8236923F00403F7
S315080026FC2361E5E7781F002000200240124BDB68B7
S3150800270C13F0100305D011491023CA6942F00202CE
S3150800271CCA610D4AD268500706D50C4943F0040322
S3150800272CCA6942F00102CA61074AD169C90708D5C4
S3150800273C0648C16941F00401C161D16921F0010162
S3150800274CD161014AD360704700200240781F0020EF
S3150800275C064B186910F0800006D00549054A5960E1
S3150800276C5A601869C0F3C010704700BF00200240B9
S3150800277C23016745AB89EFCD034A0020136943F063
S3150800278C80031361704700BF0020024070B50446F1
S3150800279C01F0FAFD124D064601E0621C13D1EB68F6
S315080027AC0F4ADB07F9D4D368980644BF2023D360B5
S315080027BC0B4BDA68D10602D4DA69D2070BD5FFF7C8
S315080027CC9DFF012070BD24B101F0DEFD801B844203
S315080027DCE5D2032070BDD86810F00400EFD170BDA7
S315080027EC002002402DE9F84FDFF8A08098F8184031
S315080027FC012C02D10220BDE8F88F1E46044601239F
S3150800280C4CF2503091468B4688F81830FFF7BEFFCD
S3150800281CA0BB012C37D0022C0CBF02200420471E6B
S3150800282CFFB20137DFF868A000253F01C5F1200289
S3150800283C0023C8F81C3006FA02F229FA05F0A5F1AD
S3150800284C2001104326FA01F1DAF81020084342F069
S3150800285C010284B2CAF810204CF25030ABF8004092
S3150800286CFFF794FFDAF81020103522F001020BF16D
S3150800287C020BCAF8102008B9BD42D7D1002388F834
S3150800288C1830BDE8F88F2046C9E700BF781F00202E
S3150800289C002002404FF6FF0206490002CB6800F4FE
S315080028ACE0601A4042F0BF6343F400330343CB6045
S315080028BC704700BF00ED00E0194B30B4DB68C3F37A
S315080028CC0223C3F10705042D03F1040428BF0425CC
S315080028DC062C18D9033B01249C40013C22400124B8
S315080028ECAC40013C214001FA03F3002842EA0302FA
S315080028FC0CDB120100F16040D2B200F5614080F8A1
S3150800290C002330BC704700221346E8E7054B00F05D
S3150800291C0F001201D2B203441A7630BC704700BFBE
S3150800292C00ED00E0FCEC00E00138B0F1807F0DD240
S3150800293C30B4074B074CF0255860002284F8235016
S3150800294C0721104630BC9A60196070470120704701
S3150800295C10E000E000ED00E010B5064B4FF0FF323A
S3150800296C0024DA601C61DA60DC60FDF7E1FF2046C2
S3150800297C10BD00BF001002400E4A38B511784FF44E
S3150800298C7A73B3FBF1F30C4A05461268B2FBF3F003
S3150800299CFFF7CAFF08B90F2D01D9012038BD044627
S315080029AC024629464FF0FF30FFF786FF034B2046B9
S315080029BC1D6038BDCC040020C4040020C8040020C7
S315080029CC074A08B51368032043F010031360FFF792
S315080029DC61FF0020FFF7D0FFFDF73AFF002008BD86
S315080029EC0020024070B50B4DE86001F0BFFC00F109
S315080029FC320605E001F03EFA01F0B8FC864207D330
S31508002A0CA868044B10F00104F4D0D868C0B270BDA5
S31508002A1C204670BD0038004038B501F0A7FC00F51B
S31508002A2CFA7503E001F0A2FC854209D9FF20FFF7ED
S31508002A3CD9FF044601F01EFAFF2CF3D1012038BD4C
S31508002A4C002038BD70B5094D04266E61FF20FFF7CE
S31508002A5CC9FFFFF7E1FF10B10124204670BD0446FB
S31508002A6C2E61FF20FFF7BEFF204670BD0014014003
S31508002A7C38B50D46010604460AD4254B04221A61BC
S31508002A8CFF20FFF7AFFFFFF7DDFF58B9FF2038BD72
S31508002A9C00213720FFF7ECFF012800D938BD04F0D8
S31508002AAC7F04EAE744F04000FFF79CFF280EFFF787
S31508002ABC99FFC5F30740FFF795FFC5F30720FFF706
S31508002ACC91FFE8B2FFF78EFF2CB1082C16D18720A0
S31508002ADCFFF788FF02E09520FFF784FF0A24FF2002
S31508002AECFFF780FF054601F0C5F92A0604F1FF3306
S31508002AFC02D513F0FF04F2D1284638BD0120FFF7A2
S31508002B0C71FF0C2CEAD1FF20FFF76CFFE6E700BF3C
S31508002B1C0014014038B505460C46FFF77DFF00B991
S31508002B2C38BD2046FFF75EFFFD2C1ED0AC1C05F207
S31508002B3C022514F8020CFFF755FF023414F8030C9F
S31508002B4CFFF750FFAC42F4D1FF20FFF74BFFFF20F5
S31508002B5CFFF748FFFF20FFF745FF00F01F00A0F125
S31508002B6C0500B0FA80F0400938BD0120D8E700BF4F
S31508002B7CF8B505460E4601F0F9FB00F1640703E0CB
S31508002B8C01F0F4FB874222D9FF20FFF72BFF0446FE
S31508002B9C01F070F9FF2CF3D0FE2C18D1AC1CFF20D9
S31508002BACFFF720FF04F8020CFF20FFF71BFF04F8C1
S31508002BBC010C01F05FF9023E04F10204EFD1FF208B
S31508002BCCFFF710FFFF20FFF70DFF0120F8BD0020CF
S31508002BDCF8BD00BF002840F0CA802DE9F04FAC4F75
S31508002BEC9BB03B7803F0020303F0FF0523B138785A
S31508002BFCC0B21BB0BDE8F08F40F2044EA54BDFF80F
S31508002C0CA8929A6906A942F008029A619A694FF045
S31508002C1C010B02F008020392039A9A69484642F09D
S31508002C2C20029A619A699C4E02F020020492049A38
S31508002C3CDA694FF0040A42F48042DA61DB6902224F
S31508002C4C03F480430593CDF818E008920192059B8E
S31508002C5C0995CDF81CB0FEF7B7FF904BC9F810A034
S31508002C6C0693092306A93046079303230893099567
S31508002C7CFEF7AAFF8A4B06A930460693CDF81CA088
S31508002C8CFEF7A2FF4FF48273DFF8248211934FF4F8
S31508002C9C007315933823404610A9169307231993E6
S31508002CAC109512951395149517951895FEF702FF1E
S31508002CBCD8F80030DFF8ECE143F04003019AC8F885
S31508002CCC00303046C9F810A00BA9CDF830B00D92DB
S31508002CDC0E95CDF82CE0FEF777FF4FF400434446EB
S31508002CEC33614FF0FF080A2601F040FB00F164053A
S31508002CFC03E001F03BFB854202D3A3689A07F8D59B
S31508002D0CC4F80C8001F032FB00F1640503E001F015
S31508002D1C2DFB854202D3A368DB07F8D5013EE3D128
S31508002D2C6048092203230BA90B905B480C920D9360
S31508002D3C0E96FEF749FF5C4B04225A613146304623
S31508002D4CFFF796FE0128044613D05849564B042221
S31508002D5C002008601A61FF20FFF744FE3B7843F019
S31508002D6C01033B703878C0B21BB0BDE8F08F012068
S31508002D7C704701F0FBFA4FF4D57100F57A75082007
S31508002D8CFFF776FE012837D10BAC26460DF1300835
S31508002D9CFF20FFF727FE06F8010BB045F8D19DF882
S31508002DAC2E30012BD1D19DF82F30AA2BCDD102E094
S31508002DBCFFF75EFE38B101F0D9FA85424FF0804133
S31508002DCC4FF0A900F4D801F0D1FA8542BDD90021FB
S31508002DDC3A20FFF74DFE0028B7D1FF20FFF702FE79
S31508002DEC04F8010BA045F8D19DF82C3013F0400FD0
S31508002DFC14BF0C24042420E03146A920FFF738FE22
S31508002E0C01289ABF0224A926264605E03046FFF774
S31508002E1C2FFE38B101F02EF801F0A8FA85424FF0D2
S31508002E2C0001F3D801F0A2FA85428ED94FF400714D
S31508002E3C1020FFF71DFE002887D11C491A4B0422C7
S31508002E4C0C60FF201A61FFF7CDFD3B78184C03F098
S31508002E5CFE033B702368082223F0400323600023FB
S31508002E6C10931293139314931793189310A907237B
S31508002E7C20464FF482764FF40075199311961595E2
S31508002E8C1692FEF717FE236843F040032360AEE65E
S31508002E9CCD04002000100240000C0140A000A00444
S31508002EAC40004004800080040014014064060020A1
S31508002EBC0038004018B9034B1878C0B27047012087
S31508002ECC704700BFCD04002038B510B10424204645
S31508002EDC38BD1C46002BF9D01D4B1B78D80701D5DD
S31508002EEC0324F4E71B4B0D461B681B0758BF5202FD
S31508002EFC012C11461ED01220FFF7BAFD58B1012439
S31508002F0C154B04221A61FF20FFF76CFDDFE700F072
S31508002F1CB1FF013C09D028464FF40071FFF728FE93
S31508002F2C05F500750028F2D1012400210C20FFF7C5
S31508002F3C9FFDE5E71120FFF79BFD0028E0D1284609
S31508002F4C4FF40071FFF714FEB0FA80F46409D7E762
S31508002F5CCD040020640600200014014010B582B090
S31508002F6C18B10424204602B010BD002BF9D00C462B
S31508002F7C2B490878C00701D50324F3E709784907D4
S31508002F8C01D50224EEE727490968080758BF5202FB
S31508002F9C012B37D011F0060F2BD1114619200093AF
S31508002FACFFF766FD009B60B101241F4B04221A61D2
S31508002FBCFF20FFF717FDD5E700F05CFF009B013BF0
S31508002FCC09D02046FC210093FFF7A4FD04F50074F4
S31508002FDC009B0028F0D10093FFF71EFD009B0028EC
S31508002FECE2D01C1C4FF0FD0018BF0124FFF7FAFCB9
S31508002FFCDBE71946972001920093FFF739FD019AF2
S3150800300C009BCAE711461820FFF732FD0028CBD1E2
S3150800301C2046FE21FFF77EFDB0FA80F46409C4E76A
S3150800302CCD040020640600200014014008B10420D9
S3150800303C7047844B1B78D80701D50320704770B5A9
S3150800304C154684B00E2900F2A480DFE801F060660C
S3150800305CA22AA2A2A2A2A2A25B4D9A1708007A4B98
S3150800306C1B685B0700F1BA800124784B04221A61AD
S3150800307CFF20FFF7B7FC204604B070BD00213A20AC
S3150800308CFFF7F6FC0028EFD16C1E0335FF20FFF77F
S3150800309CA9FC04F8010F00F0EDFEAC42F6D10024B1
S315080030ACE3E7694E336813F0040174D000218D20D0
S315080030BCFFF7DEFC0028D7D1FF20FFF793FC102181
S315080030CC6846FFF755FD0028CED03024FF20FFF7C1
S315080030DC89FC601E10F0FF04F8D19DF80A20102315
S315080030EC120993402B60C0E700210920FFF7C0FCAA
S315080030FC0028B9D128461021FFF73AFDB0FA80F41A
S3150800310C6409B2E7504B00241B681370ADE7FFF750
S3150800311C99FCB0FA80F46409A7E700210920FFF7A7
S3150800312CA7FC044600289FD110216846FFF720FD0E
S3150800313C002899D09DF800309B09012B60D09DF88A
S3150800314C05309DF80A609DF8092003F00F019DF8DB
S3150800315C07009DF8063001EBD61152009DF8086061
S3150800316C023102F0060280009B020A4403F4406313
S3150800317C00EB9611D2B20B44093A013393402B60FB
S3150800318C73E700210A20FFF773FC00287FF46CAF65
S3150800319CB0E7042469E70920FFF76AFC044600280F
S315080031AC7FF462AF10216846FFF7E2FC00283FF473
S315080031BC5BAF336813F0020332D09DF80A309DF8E2
S315080031CC0B105B009DF80D2003F07E0303EBD11367
S315080031DC92090133013A93402B6046E700218D2072
S315080031ECFFF746FC00287FF43FAFFF20FFF7FAFBFA
S315080031FC28464021FFF7BCFCB0FA80F4640934E792
S3150800320C9DF807309DF808101B049DF8092003F457
S3150800321C7C13013302EB012213449B022B6024E737
S3150800322C9DF80B409DF80A20E00000F01800C2F348
S3150800323C840100EB54104A1C00FB02221C462A602F
S3150800324C13E700BFCD0400206406002000140140DB
S3150800325C014B1880704700BF6C06002010B501F0B2
S3150800326C85F80E4C236898420DD30D4B1A785AB133
S3150800327C0C4A002020211870516101F077F80A4B8E
S3150800328C1B881844206010BD02F1804202F5843276
S3150800329C0120202118701161EFE700BF6806002095
S315080032AC6E060020000801406C060020014B202207
S315080032BC5A61704700080140034B4FF480520128AD
S315080032CC0CBF5A611A61704700100140704700BF65
S315080032DC704700BF08B5054B9B68DB0701D4002077
S315080032EC08BDFFF7E3FF012008BD00BF0008014039
S315080032FC6420FFF7ADBF00BFFFF7B0BF00B5C7B07E
S3150800330C002168464FF48C72FCF750FF6946094851
S3150800331C02F0F8FF50B9009828B19DF8080080F023
S3150800332C1000C0F3001047B05DF804FB002047B04E
S3150800333C5DF804FBA466000800487047A4660008FC
S3150800334C10B5074C002320460A22064984F8283271
S3150800335C02F060FC10B9012384F8283210BD00BFB6
S3150800336C70060020C466000808B5084890F828328C
S3150800337C012B04D0BDE80840054802F0F3BF02F063
S3150800338CFDFEBDE80840024802F0ECBF70060020BE
S3150800339CA4660008034890F82832012B00D0704721
S315080033AC02F0ECBE7006002010B5094C94F82832D1
S315080033BC012B00D010BD214603F058F80028F9DA85
S315080033CC002384F828322046BDE8104002F0D6BE09
S315080033DC70060020054B00221A709A6483F8422066
S315080033ECA3F844209A705A70704700BF9C080020B6
S315080033FC024B1878003018BF012070479C08002033
S3150800340C024B002283F84220704700BF9C0800201C
S3150800341CF8B50578FF2D41D0B74C2378012B00D091
S3150800342CF8BDC93D0646352D00F24A81DFE815F090
S3150800343C17014801480191004801480199007D008F
S3150800344CA100AE004801480148014801480148015D
S3150800345C480148014801480148014801480148010A
S3150800346C48014801480148014801480148014801FA
S3150800347C48014801480148014801480148014801EA
S3150800348C48014801BD00D800E5002F014801480154
S3150800349C480137014801F90001010E0100F09EF9B7
S315080034AC954CE8B9FE2110220223E1702271A4F88A
S315080034BC443094F84230904A012B09D0B2F84410A3
S315080034CC012384F842308D48BDE8F84000F0FEBC74
S315080034DCFE2210230221E2702371A4F84410EFE7B0
S315080034EC002310220126637063712271E570267021
S315080034FC00F00CFDA07100F0FBFCE07100F0F8FC8C
S3150800350C0823D84020726672A672A4F8443000F0DC
S3150800351C4BFF94F84230784A012BD9D0B2F94410B3
S3150800352C00297FF77DAF89B2CAE700F0EFFC737804
S3150800353C0138984259DDFF220123E270A4F8443081
S3150800354C71786D4D002940F0C88000F037FF0028CF
S3150800355CDFD1FE2131220223E1702271A4F8443016
S3150800356CA7E701F0C9F8FF220123E270A4F844305A
S3150800357C9FE74168A06C604D00F01AFF0028E8D060
S3150800358CFF220123EA70A5F8443092E70025FF23B1
S3150800359CE3702571657100F0B9FC0723A071E5711C
S315080035AC25726572A4F8443083E7FF23E3704668F6
S315080035BCA76C002E00F09D80002517F8013B1D44D2
S315080035CC00F058FC013EEDB2F7D100230121082288
S315080035DCC4F8075021716371A371A4F8442068E7F5
S315080035EC00F094FC7378984272DCFE2122220223A6
S315080035FCE1702271A4F844305BE700F087FC72781E
S3150800360C9042F2DDA16C3E4801F098F8FF23E37076
S3150800361C7378A26C1344A36473780133A4F844300A
S3150800362C77E7FE2100220223E1702271A4F84430C8
S3150800363C3FE760780023FF2106226071E170237151
S3150800364CA371E3712372A4F8442032E70023FF2107
S3150800365C012223706370E170A4F8442029E7A56C55
S3150800366C00F054FC721C411E2846234D00F09EFEA9
S3150800367C00283FF46EAFFF23EB7000F047FCAB6CF1
S3150800368C013803440122AB64A5F8442011E7FF2353
S3150800369CE37042680123A264A4F8443009E7194D83
S315080036AC0023FF2007210822A564E07023716371AB
S315080036BCA37123726372A372E171A4F84420F8E62D
S315080036CCFE2120220223E1702271A4F84430F0E690
S315080036DC71680B48A164727896E7B21CA86C00F066
S315080036EC65FE00283FF435AF7378AA6C1344AB64B7
S315080036FC0FE7354669E700BF9C0800209F080020A5
S3150800370CA0080020D4660008092800F00F0302D987
S3150800371C03F13700704710B503F1300402F04EFF81
S3150800372C2044437803F00303022B14BF2046A4F16C
S3150800373C2000C0B210BD00BF38B5054600090C46BE
S3150800374CFFF7E2FF207005F00F00FFF7DDFF0023FF
S3150800375C6070A370204638BDF8B50026471E451C78
S3150800376C17F8014F02F02AFF2044437803F00303AD
S3150800377C022B08BF203CE3B2A3F13002D2B2162AC0
S3150800378CA3F13A010DD806290BD9092A84BF373B70
S3150800379CDAB202EB0613AF4203F0FF06E0D130466D
S315080037ACF8BD0020F8BD00BF10B50023074C1A461B
S315080037BC07490848237002F0FFF900B910BD7721B4
S315080037CC0548BDE8104000F009BC00BF28090020D8
S315080037DCDC66000834090020E0660008024B1878FD
S315080037ECB0FA80F0400970472809002010B500F09F
S315080037FC8FFB012802D0054C23780BB1002010BD95
S3150800380CFFF77CFD0128F9D1207010BD280900208E
S3150800381C38B50546047802F0D1FE2044437803F007
S3150800382C0303022B08BF203C532C01D0032038BDC0
S3150800383C02F0C4FE6B78184442785207F6D5312B41
S3150800384C05D0322B05D0332BF0D1022038BD002001
S3150800385C38BD012038BD00BF70B506460230FFF7EB
S3150800386C7BFF0546043684B23046FFF775FF013CEC
S3150800387CA4B22844012CC5B206F10206F4D8304687
S3150800388CED43FFF769FFEDB2281AB0FA80F040094C
S3150800389C70BD00BF2DE9F041044616460F460029B7
S315080038AC49D0002847D02046FFF7B2FF0328054623
S315080038BC3ED02046FFF7D0FF002800F09280012D5D
S315080038CC3FD06BD3022D33D1A01CFFF745FF05461D
S315080038DC201DFFF741FF00063860A01DFFF73CFFCF
S315080038EC3B6804F10C0803EB0040386004F108004F
S315080038FCFFF732FF3B6803EB0020386004F10A003F
S3150800390CFFF72AFF3B686C1F184424B2386066B16F
S3150800391C002C0ADD00254046FFF71EFF6B1C705570
S3150800392C9DB2A54208F10208F5DB2046BDE8F081F8
S3150800393C0020BDE8F08140F261212C4800F04EFBD6
S3150800394CB1E7A01CFFF708FF0546201DFFF704FF8B
S3150800395C00043860A01DFFF7FFFE3B6804F10A0857
S3150800396C03EB0020386004F10800FFF7F5FE3B680E
S3150800397C2C1F184424B23860002ED6D0002CD4DD67
S3150800398C00254046FFF7E8FE6B1C70559DB2A54214
S3150800399C08F10208F5DB2046BDE8F081A01CFFF70C
S315080039ACDBFE0546201DFFF7D7FE00023860A01D7A
S315080039BCFFF7D2FE3B68033D18442DB20834386035
S315080039CC66B1002D0ADD00272046FFF7C5FE7B1CD5
S315080039DCF0559FB2AF4204F10204F5DB2846BDE868
S315080039ECF0814FF0FF30BDE8F08100BFE0660008BB
S315080039FC2DE9F843AA4F3C783CB1012C00F017810D
S31508003A0C022C00F08E80032C01D0BDE8F883A54E5D
S31508003A1CA54D06F50C7228464FF4807102F0FCFC95
S31508003A2C96F84192B9F1000F40F0BB81002855D0A9
S31508003A3C05F5807205F5C0712846FFF72BFFB0F126
S31508003A4CFF3F804600F01E81002847DD9748FFF7A8
S31508003A5CABFC43469649974AA2FB0303DB0801F1E4
S31508003A6C0101F9D1444693480B70A0FB0423DB08EB
S31508003A7C03EB8302A4EB4202303201F8012D1C46FB
S31508003A8C002BF2D18A48FFF78FFC8B48FFF78CFC8A
S31508003A9C874995F88301FFF74FFE884995F8820107
S31508003AACFFF74AFE864995F88101FFF745FE8549D9
S31508003ABC95F88001FFF740FE7D48FFF775FC8248B4
S31508003ACCFFF772FC4146D5F88001804A00F06EFC7F
S31508003ADC002800F079817E48FFF766FCD6F8442268
S31508003AECD6F83C329A4290D17A48FFF75DFC00F042
S31508003AFC65FC0446002800F080817548FFF754FCE5
S31508003B0C7548FFF751FC754802F038FB7448FFF707
S31508003B1C4BFC00233B70FFF727FCBDE8F84300F08D
S31508003B2CEBBD604E604D06F50C7228464FF480715D
S31508003B3C02F072FC96F84192B9F1000F40F03F8101
S31508003B4CD0B14A4605F5C0712846FFF7A3FEB0F179
S31508003B5CFF3F804600F05D8100280DDD614C6368EF
S31508003B6C002B00F019812268D5F880111A4491426D
S31508003B7C40F0CA8003446360D6F84422D6F83C3237
S31508003B8C9A427FF442AF0021544802F009FB002800
S31508003B9C40F04D81534C6368002B41D04C48FFF7DD
S31508003BAC03FC5148FFF700FC636841491A46414833
S31508003BBCA0FB0252D20801F10101F9D13D4D0A7060
S31508003BCCA5FB0302D20802EB8200A3EB40033033B9
S31508003BDC01F8013D1346002AF2D13548FFF7E4FBFC
S31508003BEC4248FFF7E1FB3249E078FFF7A5FD334978
S31508003BFCA078FFF7A1FD32496078FFF79DFD3149A2
S31508003C0C2078FFF799FD2A48FFF7CEFB2E48FFF7D9
S31508003C1CCBFB94E8030000F0CBFB002800F0E08017
S31508003C2C2B48FFF7C1FB03233B70BDE8F88300F074
S31508003C3CBBFBFFF785FB2E48FFF7B6FB2D48FFF7B6
S31508003C4CB3FBFFF779FB22460146244801F0E2FF55
S31508003C5C054638B12848FFF7A7FB2046BDE8F843C8
S31508003C6CFFF798BB1A48FFF79FFB2448FFF79CFB06
S31508003C7C2348FFF799FB1B4B02221D605D603A70C7
S31508003C8CBDE8F8831F48FFF78FFB2046FFF782FB3A
S31508003C9C06F50C7002F072FA87F80090BDE8F88306
S31508003CAC28090020340900208C0D0020186800080B
S31508003CBCE8080020CDCCCCCC28680008EA080020FF
S31508003CCCEC080020EE080020586800088C0E00202E
S31508003CDC4C670008406800085C680008640B002004
S31508003CEC746800082C090020A8670008B467000847
S31508003CFCF86600081C670008446700085467000843
S31508003D0C78670008F46700084B48FFF74DFB4B48EB
S31508003D1CFFF74AFB63684A491A464A48A0FB02E27F
S31508003D2CD20801F10101F9D1DFF818E10A70AEFBEE
S31508003D3C0302D20802EB8200A3EB4003303301F8EE
S31508003D4C013D1346002AF2D13D48FFF72DFB3E48AC
S31508003D5CFFF72AFB3A49E078FFF7EEFC3B49A078D7
S31508003D6CFFF7EAFC3A496078FFF7E6FC3949207810
S31508003D7CFFF7E2FC3248FFF717FB3748FFF714FB4F
S31508003D8C94E80300354C00F013FB48B32A48FFF7B8
S31508003D9C0BFB3348FFF708FBD5F8803184E808019C
S31508003DACEAE63048FFF700FB0220FFF7F3FA06F5C0
S31508003DBC0C7002F0E3F900233B70BDE8F8832A483F
S31508003DCCFFF7F2FA2046F0E72748FFF7EDFA062048
S31508003DDCFFF7E0FA254802F0D1F93C70BDE8F88304
S31508003DEC2148FFF7E1FA0520FFF7D4FA1F4802F03D
S31508003DFCC5F900233B70BDE8F8831B48FFF7D4FAD6
S31508003E0C0720FFF7C7FA194802F0B8F93C70BDE865
S31508003E1CF8831548FFF7C8FA0320FFF7BBFA06F52F
S31508003E2C0C7002F0ABF987F80090BDE8F8830E48E1
S31508003E3CFFF7BAFA0420D7E74C670008A86700080A
S31508003E4CE8080020CDCCCCCCB4670008EA080020E2
S31508003E5CEC080020EE080020586800082C09002001
S31508003E6C78670008D067000844670008640B0020D0
S31508003E7CFFF73EBAFFF740BA08B5FFF7ABFA00F002
S31508003E8C03F9024B02221A7008BD00BFCE040020AB
S31508003E9C00B583B00DF10701094800F087F9012830
S31508003EAC02D003B05DF804FB064B02229DF80710FE
S31508003EBC03481A70FFF7ACFA03B05DF804FB00BFB1
S31508003ECC100F0020CE04002000F032B908B5074BBD
S31508003EDC1B78022B03D0BDE80840FFF791BAC9B28C
S31508003EEC00F034F9BDE80840FFF78ABACE04002082
S31508003EFC044B1B78032B9ABF034A32F813003F2056
S31508003F0C704700BFCE040020A0680008FFF7F0BF7A
S31508003F1CFFF76EBA08B500F0EDFBFFF7A9FF00F046
S31508003F2CFDF900F041FAFFF73FFCFFF7A5FFBDE8E6
S31508003F3C084000F037B800BF08B5FFF79BFF00F044
S31508003F4C07FAFFF755FDFFF7A3FFBDE8084000F099
S31508003F5C01B800BF10B5FFF7DBFF012806D0FFF745
S31508003F6C3DFC18B10C4C2378012B00D010BD00F089
S31508003F7CFDF90A4A0A4B12681B68134403F5FA73CF
S31508003F8C9842F3D300232370FFF730FC0028EDD1B9
S31508003F9CBDE8104000F0B0BB540F0020500F0020B5
S31508003FAC580F002008B5054B01221A7000F0DEF9EF
S31508003FBC034B1860BDE80840FFF7CCBF540F002030
S31508003FCC580F0020014B1860704700BF500F002097
S31508003FDC014B1868704700BF500F002008B5FFF753
S31508003FEC49FFFCE7012838B504460D4604D94FF4B9
S31508003FFCDE710F48FFF7F2FF04EB44040D48E400AA
S3150800400C0319597C1A7C914210D0DA681570DA6853
S3150800401C597C5D6801320131AA425974DA6003D9B8
S3150800402C02590120DA6038BD012038BD002038BDA0
S3150800403CA8680008A00F0020012870B504460E4693
S3150800404C04D94FF4EF710E48FFF7C8FF04EB44048C
S3150800405C0C4DE4002B19587C80B19A681278327092
S3150800406C9A68597C586801320139824259749A60A7
S3150800407C03D92A5901209A6070BD012070BD00BF72
S3150800408CA8680008A00F00202248F8B5224B234D3B
S3150800409C00F14006224F002103F118025E60214C04
S315080040AC461C4FF0010E5A619E60DE601E60396038
S315080040BC6E1C05F140024027DA6199740A46D962EA
S315080040CC597483F829101E625E629E6183F82AE091
S315080040DC1F7483F8287001701349204685F800E090
S315080040ECFCF7D6FE11492046FCF7FAFE2046FCF7EB
S315080040FCFFFED4F82002FDF7C7FEFFF769FFB0F5FF
S3150800410CFA6F00D3F8BD4FF4FA60BDE8F840FFF734
S3150800411C59BF00BF7C120020A00F0020D00F002032
S3150800412C9C0F0020141000202C0400208C04002066
S3150800413C10B5054CD4F82002FDF7BAFE2046BDE8AA
S3150800414C1040FCF7BBBE00BF141000203F2970B509
S3150800415C0D46044621D8134E29463078FFF742FF00
S3150800416C012803D0B9211048FFF738FFADB29DB12D
S3150800417C013DADB22544013CFFF77CFE14F8011F46
S3150800418C3078FFF72FFF01284FF0C201064801D0FF
S3150800419CFFF724FFAC42EFD170BDB5210248FFF7FB
S315080041AC1DFFD8E77C120020A86800082DE9F84303
S315080041BC1E4B1F4D0746D3F820028846FDF722FFF3
S315080041CC2C785CB91B4B1C4E18783146FFF734FF1C
S315080041DC012823D000242046BDE8F883174E154B3A
S315080041EC3178DFF85490013149441878FFF724FFE9
S315080041FC0128EFD1337899F800200133DBB29A42C3
S3150800420C3370E7D1044609F10101384600F096FAF5
S3150800421C3278002388F800202B70DCE73378013BD2
S3150800422C3E2BD7D8054B28701C70D4E714100020E9
S3150800423CBD120020D00F00205C0F00207812002041
S3150800424CF0B5194F83B03C78012C04D94FF4FF71A3
S3150800425C1648FFF7C3FE164B04EB440403EBC404E1
S3150800426C667CFEB1402E134D28BF402600240DF166
S3150800427C07013878FFF7E0FE012804F101044FF432
S3150800428CA1710A4801D0FFF7A9FE9DF80720E3B2F1
S3150800429C9E4205F8012FEAD83346074A812107487A
S315080042ACFCF7D0F903B0F0BD7C120020A868000812
S315080042BCA00F0020371200203812002014100020FE
S315080042CC70B50546FCF764FA294604461048FCF70F
S315080042DCD5F980B290B1451EADB20E4E2544013CBF
S315080042EC14F8011F3078FFF77DFE01284FF4B271E0
S315080042FC094801D0FFF772FEAC42F1D1FCF748FA37
S3150800430CBDE870400246402301210148FCF7A8B9D4
S3150800431C14100020D00F0020A868000810B4064B13
S3150800432C064C0749002205201A605C609A6010BC8E
S3150800433C18600A60704700BF10E000E03F190100E2
S3150800434CC0120020014B00221A60704710E000E0F2
S3150800435C044B1B68DB0303D5034A1368013313604C
S3150800436C704700BF10E000E0C0120020044B1B6829
S3150800437C13F4803F034B18681CBF01301860704754
S3150800438C10E000E0C0120020044B1B6813F4803FB9
S3150800439C034B18681CBF01301860704710E000E02A
S315080043ACC0120020704700BF00F0C4B800F0C4B8B3
S315080043BC00F0EEB800F058B900F098B908B500F05E
S315080043CC2FF900B908BDBDE8084000F075B900BF63
S315080043DC2DE9F84380460024FEF7BAF906E0A359FE
S315080043EC9D421AD1B7F5007F3C461CD0D8F8006020
S315080043FC271D58F8075004EB0609FFF73BFD2A461C
S3150800440C494600230220FEF7EDF90028E7D00024E0
S3150800441CFEF7B2F92046BDE8F8830446FEF7ACF978
S3150800442C2046BDE8F8830124FEF7A6F92046BDE828
S3150800443CF88300BF38B5104B0D46984219D00F4A71
S3150800444C914208D00446FFF7C3FF10B1C5F3080321
S3150800445C13B1002038BD1C462368AB4207D0204652
S3150800446C294640F8045B4FF4007200F067F92046C1
S3150800447C38BD034CEAE700BFC412002000800008D0
S3150800448CC81400202DE9F8430C46016824F4FF787B
S3150800449C1D464B1C0746164628F0010832D088459F
S315080044AC06D038464146FFF7C5FF074638B30168BC
S315080044BC641A3C44043408F5007807F1040905E04D
S315080044CC16F8013B013D04F8013B15D0FFF7D2FC69
S315080044DCC9EB0403B3F5007FF2D338464146FFF720
S315080044ECA9FF074600F1040948B14C4616F8013BEA
S315080044FC013D04F8013BE9D10120BDE8F883002011
S3150800450CBDE8F883814649F8048B414648464FF482
S3150800451C007200F013F93968C1E700BF0349044A71
S3150800452C4FF0FF330B601360704700BFC8140020B0
S3150800453CC4120020FFF7F2BF30B4104C4B1E241ADD
S3150800454CA34214D80E4B984211D90C4D431E0B445A
S3150800455CAB420CD820F4FF730A4C23F00103A34298
S3150800456C0B46014606D030BC0748FFF78BBF002028
S3150800457C30BC7047054830BCFFF784BFFFFF010805
S3150800458CFF7F000800800008C8140020C412002011
S3150800459C30B5214A4C1E121A87B000239442019357
S315080045AC31D820F47F721D4C22F00302A2422AD97C
S315080045BC194D441E0C44AC4225D80D18AD1AC5F33A
S315080045CC0903C5F38F250BBB00240123049202941F
S315080045DC0593FEF7BDF835B91BE0049B954203F528
S315080045EC8063049315D9FFF745FC01A902A8FEF7C9
S315080045FC21F80134A2B20028EFD00024FEF7BCF84B
S3150800460C204607B030BD184607B030BD0135ADB2EF
S3150800461CDAE70124F2E700BFFFFF0108FF7F000875
S3150800462C0F4B1A68013218D030B599685C68DD688A
S3150800463C18690C442C445969044498690C44D96982
S3150800464C231883B00B4402AA5B4242F8043D0421AA
S3150800465C0448FFF771FF03B030BD0120704700BF57
S3150800466CC41200200C8100080E490F4B0F4A08682B
S3150800467C1B6810B412680E4C0C31034409680D48BB
S3150800468C134422680B4401681344A2680B44D0F8FF
S3150800469CF8101344CB4200F1F80010BC0CBF0120F3
S315080046AC0020704700800008048000080880000875
S315080046BC10800008148000080A4808B503680133FE
S315080046CC02D0FFF785FE58B107480368013305D0B9
S315080046DCFFF77EFE003018BF012008BD012008BD7B
S315080046EC08BD00BFC4120020C8140020004870473B
S315080046FC0080000800F034B810B5FFF75BFE00B96F
S3150800470C10BDFEF7E7FD0028FAD0FFF7DDFBFFF733
S3150800471C19FEFEF721F9FFF74FFE074B20F0604014
S3150800472C20F07F009860FFF747FE446800F01AF8FF
S3150800473C2346BDE81040184700ED00E072B170B58D
S3150800474C0D46561EB6B20644441E15F8013B04F82F
S3150800475C013FFFF78FFBB442F7D170BD704700BF1E
S3150800476C72B6704762B670470168F1B110B40C782E
S3150800477C1F2C09D93A2C14D00A4601E03A2B06D03C
S3150800478C12F8013F1F2BF9D8002010BC70470131D5
S3150800479C8A4206D1302C04D10132026010BC0020AA
S315080047AC70474FF0FF3010BC70474FF0FF30704722
S315080047BC58B110B5036882B004460BB11A7842B9E1
S315080047CC00230B60092002B010BD00230B600920E2
S315080047DC7047D888A2889042F2D158780191FEF792
S315080047EC69FB10F001000199EAD123680B60EAE72E
S315080047FC01380A4411F8013B914200F8013FF9D1FE
S3150800480C704700BFF8B5C46A00F130070546224662
S3150800481C394640780123FEF7A1FBB0B92A6AAB6981
S3150800482CA21A9A42E8700ED2AE78012E01D80AE086
S3150800483CAB691C44013E2246012339466878FEF7CB
S3150800484C8DFB012EF4D10020F8BD0120F8BD00BF68
S3150800485C38B5C36A8B4217D0C37804460D4673B96C
S3150800486C2A46012304F130016078FEF72DFB002857
S3150800487C16BF4FF0FF3500200120E56238BDFFF763
S3150800488CC1FF0028ECD038BD002038BDF8B5C37878
S3150800489C05465BB92B78032B0DD000226878114698
S315080048ACFEF7C4FB003018BF0120F8BDFFF7AAFFBE
S315080048BC0028EFD0F8BD2B79012BEED105F130018C
S315080048CC0B4605F50C70002203F8012B83424FF0BA
S315080048DC0004F9D12B69E8681F0A1E0CEA6985F8E9
S315080048EC18321B0E4FEA102E85F8197285F81A62C3
S315080048FC070C060E85F81B3285F81C02AA235520D0
S3150800490C013285F81E7285F81F625227612685F8D2
S3150800491C2E0285F82F324120722385F8330085F84C
S3150800492C160285F8143285F8153285F81DE2EA6206
S3150800493C85F8307085F8317085F8326085F817621D
S3150800494C01236878FEF70AFB2C71A6E700224FF0C4
S3150800495CFF3310B5C270C3620446FFF779FF08B17E
S3150800496C042010BD4AF6552294F82F1294F82E32CC
S3150800497C43EA0123934201D0032010BDB4F8681012
S3150800498C94F8673094F8662043EA012342EA032335
S3150800499C0A4923F07F438B42EFD0B4F8840094F88D
S315080049AC833094F8822043EA002342EA032323F057
S315080049BC7F438B4214BF0220002010BD4641540091
S315080049CCF0B5002385B00B600F461446FFF7CCFEF6
S315080049DC061E18DBC34B53F82650BDB13D602B7829
S315080049EC04F0FE0423B16878FEF764FAC70710D5FD
S315080049FCF0B2002368702B70FEF7ECF8C60711D5D9
S31508004A0C032005B0F0BD0B2005B0F0BD0C2005B099
S31508004A1CF0BDCCB300F0040303F0FF00002BF0D07C
S31508004A2C0A20EEE70CB14107FAD400212846FFF715
S31508004A3C8DFF022806D0042824D0012840F2CE8007
S31508004A4C0D20DEE76C46684605F5FC7305F50E7613
S31508004A5C13F8062C42B11F8813F8012C13F8021C04
S31508004A6C42EA072241EA02221033B34240F8042BE9
S31508004A7CEED104AF54F8046B03203EB9A742F9D122
S31508004A8C0428DDD10120BCE72046BAE73146284682
S31508004A9CFFF75CFF0128F1D895F83C2095F83B30D8
S31508004AAC43EA0223B3F5007FCAD195F8471095F867
S31508004ABC463053EA012340F09380B5F8561095F822
S31508004ACC553095F8542043EA012342EA032195F818
S31508004ADC4070A9617B1E012BAF70B1D895F83D309B
S31508004AEC9AB26A81002AABD05A1E1A42A8D195F8F6
S31508004AFC412095F8424042EA042422072C819FD192
S31508004B0C95F8440095F8432052EA002209D1B5F8E5
S31508004B1C52E095F8510095F8502040EA0E2042EAEA
S31508004B2C002295F83FE095F83E0050EA0E2087D013
S31508004B3C01FB07F700EB141EBE44724580D3CEEB7F
S31508004B4C0202B2FBF3F3002B3FF47AAF40F6F57290
S31508004B5C934240F2A5804FF6F572934240F2848058
S31508004B6C95F85B7095F85A2002333044B64452EAED
S31508004B7C07226B612862C5F828E0EE617FF460AF06
S31508004B8C002C7FF45DAFB5F85E4095F85D0095F89E
S31508004B9C5C209B0040EA042003F2FF1342EA002241
S31508004BACB1EB532F6A62FFF44BAF95F8611095F889
S31508004BBC60304FF0FF3243EA0123012B4FF080019E
S31508004BCC2A61EA6029710DD00323474A2B70138892
S31508004BDC002001339BB21380EB8012E700265BE7BB
S31508004BEC194674E7711C2846FFF732FE0028EBD1EC
S31508004BFC4AF6552295F82F0295F82E32002143EAEB
S31508004C0C002393422971DFD1698E95F8312095F8E6
S31508004C1C303042EA0122354943EA02238B42D3D18A
S31508004C2CB5F8161295F8152295F8143242EA0122AF
S31508004C3C2F4943EA02238B42C6D1B5F81A6295F876
S31508004C4C1902B5F81E4295F81D1295F8182295F812
S31508004C5C1C3240EA062041EA042142EA002243EAD1
S31508004C6C01232A61EB60AFE7023330440EEB0602F0
S31508004C7C6B612862AA62EE61002C3FF4E1AE5B0020
S31508004C8C03F2FF133844B1EB532F6862FFF4D8AE26
S31508004C9C4FF0FF3380222B61EB602A71022394E7D5
S31508004CAC023330440EEB06026B612862AA62EE618F
S31508004CBC002C3FF4C5AE03F0010202F2FF1203EB1F
S31508004CCC430302EB53033844B1EB532F6862FFF4EA
S31508004CDCB7AE4FF0FF3380222B61EB602A710123AC
S31508004CEC73E700BFD0180020CC180020525261413F
S31508004CFC72724161012919D94269F8B5914208D2F3
S31508004D0C02780646022A0C462BD0032A10D0012A12
S31508004D1C01D00120F8BD016A04EB540501EB5521BD
S31508004D2CFFF796FD78B34FF0FF30F8BD01207047BA
S31508004D3C016A01EBD411FFF78BFD0028F3D1A10012
S31508004D4C01F4FE7101F13003334458885A78314422
S31508004D5C91F8303042EA002043EA002020F07040F7
S31508004D6CF8BD016A01EB1421FFF772FD0028DAD1B0
S31508004D7C610001F4FF71731893F8310093F8303021
S31508004D8C43EA0020F8BD316AC5F308036F1C3344A7
S31508004D9C01EB5721304693F83050FFF759FD0028A0
S31508004DACC1D1C7F30803334493F83000E30745EA47
S31508004DBC00204CBF0009C0F30B00F8BDB1F5001F6D
S31508004DCC01D3022070472DE9F04111F01F080C465B
S31508004DDC02D00220BDE8F0818168054604610768A7
S31508004DEC29B93B78022B1AD97B6AC3B119467E8935
S31508004DFC7602B4422AD3A41B384608E00128E8D91F
S31508004E0C7B699842E5D2A64221D82868A41BFFF7ED
S31508004E1C71FF431C0146F1D10120BDE8F0813B89A5
S31508004E2CB3EB541FD5D9D7F82480C5F81880696117
S31508004E3CB8F1000FCDD0C4F30803303708EB54246F
S31508004E4C1F44EF61AC610020BDE8F0817B69023B31
S31508004E5C8A1E9A4204D2B7F80A80BB6A02FB083843
S31508004E6CC5F81880E3E700BF2DE9F04790F80090E5
S31508004E7C0446B9F1020F0D46164657D0B9F1030F81
S31508004E8C2FD0B9F1010F03D002273846BDE8F087B9
S31508004E9C016A05EB550801EB5821FFF7D9FC0746C3
S31508004EAC0028F2D108F1010AEB07C8F30808A04458
S31508004EBC53D598F83030204603F00F0343EA06130F
S31508004ECC88F83030216A84F8039001EB5A21FFF7F1
S31508004EDCBFFC00284CD1CAF3080AA244C6F307162D
S31508004EEC52E0016A01EBD511FFF7B2FC0746002820
S31508004EFCCBD1AD0005F4FE7505F1300323445A8871
S31508004F0C26F07046120402F070421643300C254403
S31508004F1C4FEA162E310E012285F83060987083F808
S31508004F2C01E0D970E2703846BDE8F087016A01EBFA
S31508004F3C1521FFF78DFC07460028A6D16D0005F450
S31508004F4CFF756119C6F30722012381F8306081F8D1
S31508004F5C3120E3703846BDE8F08788F83060216A5E
S31508004F6C84F8039001EB5A212046FFF771FC08B12F
S31508004F7C07468AE7CAF3080AA2449AF83020C6F309
S31508004F8C032622F00F02164301238AF83060E370D9
S31508004F9C7BE700BF2DE9F04107468846066839BB12
S31508004FACF5687369EDB901252C4606E0012815D07C
S31508004FBC01302BD0AC4218D0736901349C4202D311
S31508004FCC012D12D9022421463868FFF793FE0028D2
S31508004FDCECD1012C02D973699C421BD30120BDE884
S31508004FECF0819D4228BF0125DEE70020BDE8F0814F
S31508004FFC3046FFF77FFE0128F0D9431C06D07369AB
S3150800500C9842ECD34546CFE70128E7D14FF0FF305D
S3150800501CBDE8F0814FF0FF3221463046FFF724FFFA
S3150800502C0028F1D1B8F1000F0CD0B8F1010FD5D981
S3150800503C73699845D2D2414622463046FFF714FF8B
S3150800504C0028E1D172693369023A9342F46001D2BD
S3150800505C013B33613379204643F001033371BDE8D4
S3150800506CF08100BF83690BB9042070472DE9F04F16
S3150800507C056983B02035B5F5001F03D3042003B0AA
S3150800508CBDE8F08FC5F308070E46044602681FBB39
S3150800509C41690133836129B35389013B13EA5528C6
S315080050AC1AD110460192FFF725FE01288146019A6E
S315080050BC20D9B0F1FF3F31D0536998421CD2861ED5
S315080050CC023B9E42C4F8149004D2B2F80A80936A42
S315080050DC06FB0838C4F8188030371744E761256191
S315080050EC0020CCE71389B3EB551FF5D80023A36131
S315080050FC0420C4E70220C2E7002EF7D061692046D7
S3150800510C0192FFF747FF019A814648B90720B6E78F
S3150800511C10460192FFF776FB019A48B10120AEE7DB
S3150800512C0128E7D0B0F1FF3FF8D0D378002BEFD1A8
S3150800513C02F1300302F50C70002103F8011B8342BF
S3150800514CFBD15369A9F10206023B9E4238BF936A0A
S3150800515C51892CBF002306FB01334FF0000AD3629A
S3150800516C4FF0010B0EE082F803B010460192FFF7E0
S3150800517C49FB0028D2D1019A0AF1010AD36A51894E
S3150800518C0133D3628A45EED3D16A5369CAEB01015E
S3150800519CD16295E7416A2DE9F0414B1C0446056836
S315080051AC066904D0FFF70AFE08B1BDE8F0814FF096
S315080051BCE50801270BE0E36983F80080EF702369A3
S315080051CC9E42F2D901462046FFF74CFF28B9A16941
S315080051DC2846FFF73DFB0028EDD0042808BF02201F
S315080051ECBDE8F0812DE9F04F002185B00746D0F8CF
S315080051FC0080FFF7E3FD00284FD14FF0FF334FF047
S3150800520CFF0A994656467B620AE00F2B48D0C7F828
S3150800521C2490FF2600213846FFF724FF00283CD1AE
S3150800522CB9694046FFF714FB002836D1FC69257886
S3150800523C002D00F08880E27AE52D02F03F03BB7161
S3150800524CE5D01207E1D40F2B2AD076B9214604F102
S3150800525C0B0011F8013BF20142EA56061E44814244
S3150800526C06F0FF06F5D1B24571D0396ACB7ADB0761
S3150800527CCDD420460A7810F80B3B01349B1A013121
S3150800528C002BC4D114F8013B11F8012B8442A3EB73
S3150800529C0203F5D1002BBAD1184605B0BDE8F08F3C
S315080052ACBB6A002BB6D0680649D53A6994F80DA0A6
S315080052BC05F0BF057A62627B524542D1E17EA07E3B
S315080052CC50EA012138D12078012100F03F0001383D
S315080052DC00EB400A00EB8A0A0395DFF8A0B02546D6
S315080052ECCDF800801C4601920846029713E0BAF1E5
S315080052FCFE0F1DD8304601F003F9804634F81A0023
S3150800530C01F0FEF8804513D13046BA461A4B5B4578
S3150800531C1FD01BF8011F6E187678695C0AF1010715
S3150800532C41EA06260028E2D14FF6FF739E42EDD0DD
S3150800533CDDF80080019A029F9246FF266AE7AE4284
S3150800534CB9D0FF2666E7042005B0BDE8F08F00202B
S3150800535CA3E723462C462178DDF800804906039DF1
S3150800536C019A029F04D518B133F81A30002BE3D1F1
S3150800537C013DEEB292464DE7706900086469000873
S3150800538C2DE9F04FD0F8209089B099F80B3013F02E
S3150800539CA00303D0062009B0BDE8F08FD0F828800A
S315080053ACB8F8006036B11E46434633F8022F01366C
S315080053BC002AFAD10446236805A80C22494601930B
S315080053CCFFF716FA9DF81F30DD0772D5002389F80A
S315080053DC0B300B22A36205A948460125FFF708FAEC
S315080053EC2B467E270DF1140E072203F00F0000F151
S315080053FC3001392988BF00F137011B0902F1FF3248
S3150800540C0EF8011DF1D108A9114401F8147C002AE3
S3150800541C00F0A98099F80010202908D0494603E025
S3150800542C11F8010F202802D001339A42F8D109EB62
S3150800543C030108A8072A104498BF10F8140C03F1A6
S3150800544C01038CBF20200132072B01F8010BF0D980
S3150800545C2046FFF7C7FE08BB0135642D00F0F28025
S3150800546C0B2205A94846FFF7C3F9052D2B46B9D9D2
S3150800547CA8F1020E3EF8022F002AB3D0102102F032
S3150800548C010000EB4303D80344BF83F4883383F04D
S3150800549C210301394FEA5202F1D1EBE704287FF4D4
S315080054AC7AAF9DF81F3089F80B309DF81F30C4F879
S315080054BC28809B0742D4002120464FF0010B266812
S315080054CCFFF77CFC002848D1054605E00546204632
S315080054DCFFF7C8FD002840D1A1693046FFF7B8F997
S315080054EC01210D44002838D1E3691B78E52B01D03E
S315080054FC002BEBD1AB45EAD1BBF1010B35D1A16938
S3150800550C0198FFF7A5F900287FF445AF0346E26931
S3150800551C02F1200102F8013B8A42FBD10B22216AD7
S3150800552CE069FFF765F9236AE169DB7A012203F082
S3150800553C18030B73019B0020DA702CE7424B0C36D0
S3150800554CA3FB063B00214FEA9B0B20460BF1010BF4
S3150800555C2668FFF733FC0028B6D0042808BF0720B6
S3150800556C09B0BDE8F08F134661E721692046A1EB27
S3150800557C4B11FFF723FC00287FF40DAF07463B467B
S3150800558C216A01F10B0011F8012BDD0145EA5303E1
S3150800559C1344814203F0FF03F5D14FF6FF769A4682
S315080055ACA1690198FFF754F9074600287FF4F3AE72
S315080055BC5FFA8BF808F1FF32034602EB420002EB66
S315080055CC80024FF00F00E5692049D4F828C001F194
S315080055DC0C0EE87285F80DA02F73AF76EF760120C6
S315080055EC4FF0FF090EE03CF812302F182B54180A0E
S315080055FC002B08BF33468E4502F1010278700AD09B
S3150800560C11F8010FB342EED12F188E4505F800900C
S3150800561C87F80190F4D1B34202D03CF812300BB99A
S3150800562C48F04008019A012385F800800021D370C0
S3150800563C2046FFF717FD00287FF4ADAEBBF1010B32
S3150800564CAED15CE70720A6E64FECC44E64690008A9
S3150800565C012908D9F8B505680E466B6907469942BB
S3150800566C03D30220F8BD022070475AB1012AF8D993
S3150800567C9342F6D9114628464FF0FF32FFF7F4FB52
S3150800568CB0B1F8BD284614E0314600222846FFF78B
S3150800569CEBFB0028F5D12B695A1C05D02A79013366
S315080056AC42F001022B612A716B699C4211D2264683
S315080056BC38683146FFF71EFB044650B10128D0D096
S315080056CC411C08D0012ECCD96B699E42DCD3022032
S315080056DCF8BD0020F8BD0120D3E700BF2DE9F04F37
S315080056EC0746D0F800A083B00B780D462F2B01F196
S315080056FC0101F9D05C2BF7D00021B96028781F2856
S3150800570C40F2308180B21F28BE6A2FD92F282DD09F
S3150800571C5C282BD00121A946A6F10208012400F029
S3150800572CCDFEF8B17F2809D822281BD09C4A01E067
S3150800573C984217D012F8013F002BF9D128F8020F1E
S3150800574C19F8010F631C1F2812D92F2810D05C28B2
S3150800575C0ED0B3F5807F05D001211C4600F0AEFEB5
S3150800576C0028DFD1062003B0BDE8F08F0024012302
S3150800577C2B441A781D462F2A03F10103F9D05C2A0B
S3150800578CF7D01F288CBF4FF000094FF004094CB115
S3150800579C06EB440232F8023D202B01D02E2B04D105
S315080057AC013CF7D100233380DCE73B6A002226F85C
S315080057BC142003F10B0006EB4402202103F8011B0D
S315080057CC8342FBD1B31E4FF0000801E008F1010833
S315080057DC33F8020F2028F9D02E28F7D0B8F1000F8D
S315080057EC01D049F00309134633F8022D2E2A01D0AD
S315080057FC013CF9D100239B462B46354626465C468A
S3150800580C082208F1010870B320281ED02E281AD0B9
S3150800581C944221D2B0456DD07F2875D82B2800F03C
S3150800582C8480DFF884E101E081427ED01EF8011FF6
S3150800583C0029F9D1A0F14101192900F29C804BF0FD
S3150800584C020BC0B274E0B04504D049F0030935F830
S3150800585C1800D6E794424DD30B2A70D0B0454BD0DE
S3150800586C49F0030948D91D463B6A1978E5296ED0D3
S3150800587C082A04BF4FEA8B0B5FFA8BFB0BF00C0262
S3150800588C0C2A59D00BF00301032955D019F0020F35
S3150800589C0AD10BF0030BBBF1010F08BF49F0100935
S315080058AC042A08BF49F0080983F80B903846FFF715
S315080058BC99FC3B6ADB7A002867D15A073FF553AF48
S315080058CCBB79DB064AD53B699AF80010C3F3080383
S315080058DC30335344D87E9A7E032942EA002202D0FA
S315080058ECBA6028780EE7597D1B7D43EA012342EA04
S315080058FC0342F5E70B2A22D04FEA8B0B5FFA8BFB98
S3150800590CB0460B220824A2E700210192009300F06E
S3150800591CD5FD009B019AF0B1224949F002090844C9
S3150800592C10F8800C00287FF479AF49F003095F2042
S3150800593C396A085501348AE749F00209A6E71D4673
S3150800594C3B6A49F003091A78E52A97D10B220521F7
S3150800595C19703B6A8CE749F00209E6E7052003B0A3
S3150800596CBDE8F08F38463B6A8022DA7203B0BDE890
S3150800597CF04FFFF723BAA0F16101192997BF203818
S3150800598CC0B2C0B24BF0010BD2E704287FF4EBAEE1
S3150800599C13F0040F08BF052003B0BDE8F08F00BF55
S315080059ACD0680008E4680008DC6800082DE9F843AC
S315080059BC436A064601330D461AD0836A18889C1C1E
S315080059CC90B103F5007901F11508002707E04C455D
S315080059DC0AD008F8010F34F8020B013728B1002158
S315080059EC00F06CFD0028F2D100272F440023BB756C
S315080059FC00210B46AC7D4FF02E0CF0695A1CC35C8B
S31508005A0C202B1AD0052B08BFE523092A3AD068188B
S31508005A1C43728CB9A3F14107192F0CD8F769082AD8
S31508005A2C3F7B8CBF4FF0100E4FF0080E17EA0E0F87
S31508005A3C1CBF2033DBB2837501310B2A1346DCD12C
S31508005A4C68182CB98475F3691B7B002B08BF28468C
S31508005A5C00234372F369DB7A2B72F369D88B5A7F6E
S31508005A6C197F42EA002241EA02222A60597E1A7EEE
S31508005A7C42EA0122AA80DA7D9B7D43EA0223EB8067
S31508005A8CBDE8F88368180CB980F816C080F809C008
S31508005A9C0131BCE72DE9F84FFF27044606683D4659
S31508005AAC042006E0FF2500212046FFF7DBFA002834
S31508005ABC57D1A169002958D03046FEF7C9FE0028EF
S31508005ACC4FD1E1690A78002A4AD0CB7AE52A03F045
S31508005ADC3F03A371E6D02E2AE4D023F02000082831
S31508005AECE0D00F2B46D1500637D523694F7B02F0F1
S31508005AFCBF05636291F80DE0BE45D3D1CA7E8B7E95
S31508005B0C53EA022326D10B782A4803F03F03013BBC
S31508005B1C012203EB430794464FF6FF7AD4F82890F4
S31508005B2C03EB870700F10C0809E0FE2F12D89C46F8
S31508005B3C29F81730013780452FD010F8012F8B180C
S31508005B4C93F801B08B5C43EA0B23BCF1000FECD144
S31508005B5C5345F0D07746FF25A5E7AA42A2D1C9E757
S31508005B6C04200023A361BDE8F88F0028F9D1002092
S31508005B7CBDE8F88F6DB901F10B0011F8013BEA018C
S31508005B8C42EA55051D44814205F0FF05F5D1BD4293
S31508005B9CEDD04FF0FF336362E9E70B785B0604D56B
S31508005BACFE2FD7D8002329F81730013DEDB27746DA
S31508005BBC79E700BF6469000810B584B004AB43F8F4
S31508005BCC041D0190184614460091FEF7CDFD021EE1
S31508005BDC0FDB0F4951F822300BB100201870019BCE
S31508005BEC8BB10020012C187041F8223004D004B077
S31508005BFC10BD0B2004B010BD024601A96846FEF77D
S31508005C0CDFFE04B010BD184641F82230EFE700BF9E
S31508005C1CD0180020F0B593B0019148B3002302F0D8
S31508005C2C1F06044615460360324603A901A8FEF76B
S31508005C3CC7FE08B113B0F0BD0399554A04AB0791DA
S31508005C4C07A8019911920F93FFF748FD98B90F9B76
S31508005C5C93F90B30002B55DB15F01C0F1BD09DF858
S31508005C6C223013F0110F42D16D0710D50820E1E749
S31508005C7C092013B0F0BD15F01C0FDBD00428D9D1C0
S31508005C8C07A8FFF77DFB0028D4D146F00806300795
S31508005C9C3AD4039D0DE09DF82230D90629D4AA07DB
S31508005CAC01D5DB0723D415F0080F039D01D046F068
S31508005CBC2006EA6A0E9B226263622978D87E9A7E4F
S31508005CCC032942EA002216D0A260597FDF8B0020F6
S31508005CDC1A7F2674607441EA0723E98842EA03238B
S31508005CECE3602560A1806061E06113B0F0BD072018
S31508005CFCA0E704209EE7587D197D41EA002142EA77
S31508005D0C0142E1E7062095E70E9B00224821612017
S31508005D1C59749A73DA7318740E9B202759769A75E8
S31508005D2CDA7518760E9B039DDF720E9B2A78DF7E3A
S31508005D3C997E032A41EA072723D000229A76DA7637
S31508005D4C2978032904BF1A755A750E9B002201215E
S31508005D5C1A775A779A77DA77E970002FA7D007A8B7
S31508005D6C3946ED6AFFF774FC00287FF463AF2946C1
S31508005D7C0398FEF76DFD039D013FEF60002896D052
S31508005D8C58E7597D1A7D42EA012247EA0247D4E7C9
S31508005D9CCC1600202DE9F04F1E4683B000230F4683
S31508005DAC336001A914460546FEF702FD28B9687C3E
S31508005DBC18B92B7CD80703D4072003B0BDE8F08F9D
S31508005DCC6B69EA6805F12809C3EB0208A04528BFE8
S31508005DDCA046B8F1000F3ED0C3F30801002959D1EB
S31508005DEC0199B1F80AB00BF1FF3B1BEA532B5DD0B6
S31508005DFCAA694B69A2F1020A023B9A4570D24B89F1
S31508005E0C886A03FB0A0000286AD05FEA58240BEB61
S31508005E1C000A22D00BEB04029A4288BFCBEB030490
S31508005E2C4878234652463946FDF74EF8002847D19E
S31508005E3C2B7C5A0604D5E869CAEB0000844247D87D
S31508005E4C64026B69326823442244B8EB04086B611C
S31508005E5C27443260C0D10020AFE7EA69924514D0D6
S31508005E6C2B7C5B060AD5487801234946FDF776F85C
S31508005E7C30BB2B7C019923F040032B744878012303
S31508005E8C52464946FDF720F8D0B96969C5F81CA0F1
S31508005E9CC1F30801C1F50074444528BF44462831AE
S31508005EAC294422463846FEF7A3FCCAE75BB9A8681C
S31508005EBC012815D9411C03D002460199A86198E717
S31508005ECC0120687479E7A9692868FEF713FFEFE7DC
S31508005EDC07EB40204FF400724946FEF789FCAFE702
S31508005EEC0220687469E700BF2DE9F04F1F4683B09E
S31508005EFC002388463B6001A916460446FEF758FC63
S31508005F0C28B9607C18B9227C910703D4072003B002
S31508005F1CBDE8F08F6369F34228BFDE43002E00F01C
S31508005F2C898004F128094FE0019AB2F80AA00AF10F
S31508005F3CFF3A1AEA532A0ED1002B74D1A06800280E
S31508005F4C7DD0012800F09980421C69D0A368A06115
S31508005F5C019A03B9A060237C5B0654D4A3695169E2
S31508005F6C023B02398B4280F088805089956A00FB87
S31508005F7C0353002B00F081805FEA562B0AEB0305CE
S31508005F8C36D00AEB0B03834288BFCAEB000B5B4681
S31508005F9C507841462A46FCF7E1FF002840D1E169D2
S31508005FAC491B8B455DD84FEA4B256369E2682B4440
S31508005FBC9A4238BF1A4611463A68761B2A446361D8
S31508005FCCE160A8443A6034D0C3F308000028ABD08B
S31508005FDCC0F50075B54228BF3546283020442A46F8
S31508005FEC4146FEF705FC237C43F040032374DCE7AB
S31508005FFCE36960699D4202D0E368984227D3E5615C
S3150800600CC0F30800E4E750780123E2694946FCF737
S3150800601CA5FF28B9237C019A23F0400323749DE736
S3150800602C0120607473E7A1692046FEF7B3FF0028C8
S3150800603C87D1227C42F020022274002067E7514661
S3150800604C2046FEF7A7FF00287FF47BAFF1E75078D0
S3150800605C01232A464946FCF737FF0028E0D1606938
S3150800606CCDE708EB41214FF400724846FEF7C0FB1A
S3150800607C237C23F04003237495E70220607446E7DB
S3150800608C70B50A2982B00E4605461AD06A68002AE7
S3150800609C08DB541CAB183C2C1E7305DCAB686C6017
S315080060AC0133AB6002B070BD01AB224605F10C01A1
S315080060BC2868FFF719FF019B1C1B18BF4FF0FF340C
S315080060CCECE70D21FFF7DCFFE0E700BFF0B583B086
S315080060DC01A90446FEF76CFB002846D1227C02F087
S315080060EC200303F0FF00002B3FD053060DD5019A71
S315080060FC0123507804F12801E269FCF72FFF0028E8
S3150800610C35D1237C23F040032374216A0198FEF7CA
S3150800611C9FFB50BB636ADA7A42F02002DA72A268F5
S3150800612C2168C2F30720D8769A760978032920D0F5
S3150800613CE168019D080A0022197758774FEA114E33
S3150800614C0F0E482001216126587683F81EE0DF776A
S3150800615C9A75DA759A74DA741E762846E970FEF71B
S3150800616C95FB237C23F02003237403B0F0BD012098
S3150800617CFBE7120C110A1A755975D9E710B582B0D6
S3150800618C0446FFF7A3FF08B102B010BD01A92046CB
S3150800619CFEF70EFB0028F7D1206002B010BD00BF39
S315080061AC70B582B00D4601A90446FEF701FB00281E
S315080061BC42D1607C00283FD1E368AB4204D2227CF2
S315080061CC12F0020F08BF1D46002263696261002D9A
S315080061DC34D0019A568976023BB1013B6A1EB3FB51
S315080061ECF6F1B2FBF6F28A425AD2A168002962D0BD
S315080061FCA16131BB0D466669C6F30803002B64D052
S3150800620CE269954261D0237C5B063AD404F12806F0
S3150800621C019B314658782A460123FCF755FE00287F
S3150800622C38D16669E368E5619E4268D9237CE660E5
S3150800623C43F020032374002002B070BD284602B038
S3150800624C70BDB54214D843E02046FEF7A3FE0146BE
S3150800625C00283CD04A1C1DD001291ED9019B5B691C
S3150800626C99421AD26369AE423344A161636130D252
S3150800627C237CAD1B9807E7D42068FEF73BFD014647
S3150800628CE8E7019B04F12806587831460123FCF708
S3150800629C65FE58B101206074CEE702206074CBE726
S315080062AC724213406361ED1AA169A2E7237C23F0BD
S315080062BC40032374ACE72046FEF76CFE0128014622
S315080062CCEBD0431CE6D0A06092E7E368ACE7354612
S315080062DC6369EE18C5F30800666170B101988B1EE8
S315080062EC4269023A9342D8D24289816A03FB021167
S315080062FC0029D2D001EB55257EE705467CE7002020
S3150800630C9AE700BF30B591B001900D46002205A959
S3150800631C01A8FEF755FB044610B1204611B030BD56
S3150800632C0F4A02AB019905A80F920D93FFF7D6F900
S3150800633C04460028F1D10D9B93F90B30002B0ADB90
S3150800634C002DEAD00B9BA875002BE6D0294605A88C
S3150800635CFFF72CFBE1E70624204611B030BD00BF41
S3150800636CCC16002030B59DB00190022202A901A8D6
S3150800637CFEF726FB029B069308B11DB030BD254AD5
S3150800638C03AB06A8019910920E93FFF7A7F90028FC
S3150800639CF3D10E9B93F90B30002B05DB9DF81E20D1
S315080063ACD10703D50720E8E70620E6E7029D0D99F5
S315080063BC2878CC7E8B7E032843EA04241BD0D3068C
S315080063CC09D406A8FEF7E6FE0028D6D1D4B9029859
S315080063DCFEF75CFAD1E711A8002111951394FEF784
S315080063ECEDFC0028C9D111A8FFF754FB0028D9D019
S315080063FC0428E6D0C1E7487D0B7D43EA002344EA2E
S3150800640C0344DCE70246214606A8FFF721F90028D3
S3150800641CB3D1DCE7CC1600202DE9F04180461746AF
S3150800642C054682B04E1E0024B4424FF0010212DA21
S3150800643C01AB69463846FFF7ADFC019B6A1C012B7C
S3150800644C09D19DF800300D2BEED00A2B2B7004F1D8
S3150800645C01041546E8D1002C4FF0000314BF404642
S3150800646C18462B7002B0BDE8F08100BF10B5044683
S3150800647C0846217894B00023019002930393D1B176
S3150800648C01A8FFF7FDFD14F8011F0029F8D1029A9F
S3150800649C002A0CDB01986B4604A9FFF725FD30B9D9
S315080064AC029A009B9A4202D1039814B010BD4FF081
S315080064BCFF3014B010BD0A46EDE700BF7F2811D98E
S315080064CC89B910B40D4AC72303E0802914D032F8D1
S315080064DC023F98428CB201F10101F6D104F1800019
S315080064EC80B210BC7047FF2804D8044B803833F8A8
S315080064FC10007047002070470020F2E7306A000849
S3150800650C264AB0F5805F264B38BF134670B441F661
S3150800651C7D5138BF6121043381B188420ED333F8DB
S3150800652C022C1E46D4B26518A8424FEA122207DB83
S3150800653C043372B133F8041C0029EED170BC7047D1
S3150800654C082AFBD8DFE802F00E12181B1E21242796
S3150800655C0A0006EB440336F81410DCE7A0F5E35002
S3150800656C80B2EBE7411A33F81100E7E7411A01F05C
S3150800657C0103C01A80B2E1E7103880B2DEE7203892
S3150800658C80B2DBE7303880B2D8E71A3880B2D5E764
S3150800659C083080B2D2E7503880B2CFE7306B0008AB
S315080065AC74690008034B1B68186A034B002808BF5C
S315080065BC1846704728040020D004002008B5034B61
S315080065CC1868FFF7EFFFD0F8EC0008BD2804002088
S315080065DC82B001B901A93AB143B113780B601278AC
S315080065EC101C18BF012003E0104601E06FF00100F3
S315080065FC02B0704749B1FF2A85BF8A2303600A7027
S3150800660C4FF0FF3098BF01207047084670470000CE
S3150800661CF8B500BFF8BC08BC9E467047F8B500BF75
S30D0800662CF8BC08BC9E46704745
S31508006634000000204F70656E424C542055736572F5
S315080066440000000057696E5553422042756C6B2052
S315080066544465766963650000303030303030303058
S31508006664303530430000000044656661756C74007B
S3150800667457696E5553422042756C6B20496E746592
S315080066847266616365000000757362645F636F6EAA
S31508006694662E6300000201026D61696E2E630000B6
S315080066A42F64656D6F70726F675F6F6C696D65785F
S315080066B4696E6F5F73746D33322E7372656300008F
S315080066C42F626F6F746C6F672E7478740000000005
S315080066D44F70656E424C5400303A00002E2E2F2E11
S315080066E42E2F2E2E2F536F757263652F66696C6570
S315080066F42E6300004669726D776172652075706451
S315080067046174652072657175657374206465746552
S31508006714637465640A0D00004F70656E696E6720C0
S315080067246669726D776172652066696C6520666F45
S31508006734722072656164696E672E2E2E0000000051
S315080067444552524F520A0D004F4B0A0D00000000E5
S315080067545374617274696E67207468652070726F09
S315080067646772616D6D696E672073657175656E63B1
S31508006774650A0D0050617273696E67206669726DE9
S31508006784776172652066696C6520746F2064657428
S3150800679465637420657261736520626C6F636B73DD
S315080067A42E2E2E0045726173696E67200000000064
S315080067B42062797465732066726F6D206D656D6FDE
S315080067C47279206174203078000000005265616493
S315080067D4696E67206C696E652066726F6D206669DE
S315080067E46C652E2E2E4552524F520A0D000000009B
S315080067F4496E76616C696420636865636B73756D4D
S3150800680420666F756E642E2E2E4552524F520A0D0F
S315080068140000000050726F6772616D6D696E6720C3
S315080068240000000020627974657320746F206D651A
S315080068346D6F72792061742030780000577269741C
S31508006844696E672070726F6772616D20636865632D
S315080068546B73756D2E2E2E00436C6F73696E6720ED
S315080068646669726D776172652066696C650A0D00E2
S315080068744669726D77617265207570646174652006
S315080068847375636365737366756C6C7920636F6D72
S31508006894706C657465640A0D000000000000080049
S315080068A43F0000002E2E2F2E2E2F2E2E2F536F75BF
S315080068B47263652F41524D434D335F53544D333202
S315080068C446312F7573622E6300000000222A3A3C73
S315080068D43E3F7C7F000000002B2C3B3D5B5D0000A7
S315080068E4809A45418E418F804545454949498E8F51
S315080068F49092924F994F555559999A9B9C9D9E9F54
S3150800690441494F55A5A5A6A7A8A9AAABACADAEAF54
S31508006914B0B1B2B3B4B5B6B7B8B9BABBBCBDBEBFED
S31508006924C0C1C2C3C4C5C6C7C8C9CACBCCCDCECFDD
S31508006934D0D1D2D3D4D5D6D7D8D9DADBDCDDDEDFCD
S31508006944E0E1E2E3E4E5E6E7E8E9EAEBECEDEEEFBD
S31508006954F0F1F2F3F4F5F6F7F8F9FAFBFCFDFEFFAD
S3150800696401030507090E10121416181C1E00000050
S315080069747D1D0100632C001E9601A01E5A01001FEE
S315080069840806101F0606201F0806301F0806401FA3
S315080069940606511F0700591F521F5B1F541F5D1F10
S315080069A4561F5F1F601F0806701F0E00BA1FBB1F05
S315080069B4C81FC91FCA1FCB1FDA1FDB1FF81FF91F01
S315080069C4EA1FEB1FFA1FFB1F801F0806901F080605
S315080069D4A01F0806B01F0400B81FB91FB21FBC1FAA
S315080069E4CC1F0100C31FD01F0206E01F0206E51FC5
S315080069F40100EC1FF21F0100FC1F4E210100322189
S31508006A0470211002842101008321D0241A05302C18
S31508006A142F04602C0201672C0601752C0201802CB8
S31508006A246401002D260841FF1A030000C700FC0074
S31508006A34E900E200E400E000E500E700EA00EB0014
S31508006A44E800EF00EE00EC00C400C500C900E6004B
S31508006A54C600F400F600F200FB00F900FF00D600B9
S31508006A64DC00A200A300A500A7209201E100ED0026
S31508006A74F300FA00F100D100AA00BA00BF001023FF
S31508006A84AC00BD00BC00A100AB00BB00912592255B
S31508006A949325022524256125622556255525632532
S31508006AA4512557255D255C255B2510251425342598
S31508006AB42C251C2500253C255E255F255A255425AD
S31508006AC469256625602550256C256725682564256E
S31508006AD4652559255825522553256B256A251825D4
S31508006AE40C25882584258C2590258025B103DF006F
S31508006AF49303C003A303C303B500C403A6039803FF
S31508006B04A903B4031E22C603B50329226122B100D0
S31508006B146522642220232123F7004822B000192283
S31508006B24B7001A227F20B200A025A00061001A032C
S31508006B34E0001703F8000703FF00010078010001CD
S31508006B44300132010601390110014A012E01790189
S31508006B54060180014D0043028101820182018401FC
S31508006B64840186018701870189018A018B018B01CA
S31508006B748D018E018F019001910191019301940178
S31508006B84F60196019701980198013D029B019C0123
S31508006B949D0120029F01A001A001A201A201A40156
S31508006BA4A401A601A701A701A901AA01AB01AC0189
S31508006BB4AC01AE01AF01AF01B101B201B301B3013A
S31508006BC4B501B501B701B801B801BA01BB01BC01E9
S31508006BD4BC01BE01F701C001C101C201C301C40160
S31508006BE4C501C401C701C801C701CA01CB01CA014D
S31508006BF4CD011001DD0101008E01DE011201F30150
S31508006C040300F101F401F401F8012801220212013A
S31508006C143A020900652C3B023B023D02662C3F0200
S31508006C2440024102410246020A0153024000810120
S31508006C348601550289018A0158028F015A02900178
S31508006C445C025D025E025F029301610262029401C4
S31508006C546402650266026702970196016A02622C5B
S31508006C646C026D026E029C01700271029D01730230
S31508006C7474029F0176027702780279027A027B020D
S31508006C847C02642C7E027F02A60181028202A9018B
S31508006C948402850286028702AE014402B101B2016A
S31508006CA445028D028E028F0290029102B7017B0380
S31508006CB40300FD03FE03FF03AC03040086038803F5
S31508006CC489038A03B1031103C2030200A303A303BE
S31508006CD4C4030803CC0303008C038E038F03D80371
S31508006CE41801F2030A00F903F303F403F503F603A0
S31508006CF4F703F703F903FA03FA03300420035004ED
S31508006D041007600422018A043601C1040E01CF0467
S31508006D140100C004D00444016105260400004300B0
S31508006D24504F534958002E000020202020202020B0
S31508006D342020282828282820202020202020202019
S31508006D442020202020202020208810101010101029
S31508006D541010101010101010100404040404040475
S31508006D64040404101010101010104141414141410F
S31508006D7401010101010101010101010101010101F1
S31508006D840101010110101010101042424242424201
S31508006D9402020202020202020202020202020202C1
S31508006DA40202020210101010200000000000000069
S31508006DB400000000000000000000000000000000C1
S31508006DC400000000000000000000000000000000B1
S31508006DD400000000000000000000000000000000A1
S31508006DE40000000000000000000000000000000091
S31508006DF40000000000000000000000000000000081
S31508006E040000000000000000000000000000000070
S31508006E140000000000000000000000000000000060
S31108006E2400000000000000000000000054
S30D08006E305502000831010008B3
S30908006E380D01000832
S31508006E3C00000000EC02002054030020BC030020D4
S31508006E4C0000000000000000000000000000000028
S31508006E5C0000000000000000000000000000000018
S31508006E6C0000000000000000000000000000000008
S31508006E7C00000000000000000000000000000000F8
S31508006E8C00000000000000000000000000000000E8
S31508006E9C00000000000000000000000000000000D8
S31508006EAC00000000000000000000000000000000C8
S31508006EBC00000000000000000000000000000000B8
S31508006ECC00000000000000000000000000000000A8
S31508006EDC0000000000000000010000000000000097
S31508006EEC0E33CDAB34126DE6ECDE05000B0000005C
S31508006EFC0000000000000000000000000000000078
S31508006F0C0000000000000000000000000000000067
S31508006F1C0000000000000000000000000000000057
S31508006F2C0000000000000000000000000000000047
S3150800725C0000000000000000000000208D0300085C
S3150800726C99030008A5030008C1030008DD030008FC
S3150800727CF903000815040008040309041201100197
S3150800728C00000040501DAC60000101020301000023
S3150800729C09022000010100C0320904000002FF00A7
S315080072AC0000070581024000FF070501024000FFA8
S315080072BC0A0610010000004001000000050700083E
S315080072CCED06000835070008000000000000000065
S315080072DCD5060008E1060008BD06000800000000F7
S315080072EC0000000000000000A506000800000000D1
S315080072FCB106000800A24A041000000001010400AF
S3150800730C4300000000000000000000000000000020
S3150800731C0000000000000000000000000000000053
S3150800732C4300000000000000000000000000000000
S3150800733C0000000000000000000000000000000033
S3150800734C43000000000000000000000000000000E0
S3150800735C0000000000000000000000000000000013
S3150800736C43000000000000000000000000000000C0
S3150800737C00000000000000000000000000000000F3
S3150800738C43000000000000000000000000000000A0
S3150800739C00000000000000000000000000000000D3
S315080073AC4300000000000000000000000000000080
S315080073BC00000000000000000000000000000000B3
S315080073CC4300000000000000000000000000000060
S315080073DC0000000000000000000000000000000093
S315080073EC01660008DD650008000000002C6D000829
S315080073FC2A6D00082B6D00082B6D00082B6D0008F4
S3150800740C2B6D00082B6D00082B6D00082B6D0008E2
S3150800741C2B6D00082B6D0008FFFFFFFFFFFFFFFF1A
S3150800742CFFFFFFFFFFFF00000100415343494900DE
S3150800743C0000000000000000000000000000000032
S3150800744C00000000000000000000415343494900B9
S3150800745C0000000000000000000000000000000012
S3110800746C00000000000000000000000006
S70508000341AE
